:08000000FC7F00208971000063
:100400000000000000000000FFFFFFFFBE03FFFF31
:100410007FB5422306A88DF81030002340F8143D24
:1004200006F0D0FB012804D1612014210C2203F036
:100430005FF907B05DF804FB0149182202F099BD8D
:10044000C073000038B548F204001249124D18225A
:1004500004F00FFC002812DA04200E49182204F0E0
:1004600008FC0028A8BF00240BDA0A48FFF7E4FFC5
:1004700028680A49402202F07CFD002038BD4FF474
:10048000004444F01C002968402204F0F2FB20469E
:1004900038BD00BF3584FF1F1482FF1F1074000099
:1004A00008B5144B202818800BD002D8E0B10828DA
:1004B00005E0802818D0B0F5807F0AD0402818D1F8
:1004C00012E0612041F270710622BDE8084003F09D
:1004D0000FB9062261204FF4966103F009F9064B2B
:1004E0001A78064B1A7008BD6120BDE8084003F079
:1004F00039B908BD4082FF1F3484FF1FFC81FF1FF4
:1005000070B5012886B0264C264E1ED126491822E9
:10051000684602F02EFDFFF795FF23490546182295
:10052000206802F026FD33685B899B071AD504A971
:1005300004221E4802F01DFD03A904221C4802F0FB
:1005400018FD1C4802A904220AE0FFF77BFF0546BC
:1005500019480422011F02F00CFD206812491822DC
:1005600002F007FD21681548182202F002FD2068FC
:1005700031681830402202F0FCFC2068037E152B05
:100580000AD00F494022183002F0F3FC054B0C4909
:100590001868402202F0EDFC284606B070BD00BF8E
:1005A0001882FF1F1482FF1F3584FF1F4584FF1F21
:1005B0004184FF1F3D84FF1F4984FF1F4D84FF1F9F
:1005C00010740000074B084A1978117018B10228FE
:1005D00004D102F0B3BA054A127800E0FF221A7083
:1005E000704700BFFC81FF1FF081FF1F3484FF1F95
:1005F000024B1A78024B1A70704700BFF081FF1F40
:10060000FC81FF1F30B51F4B1F4D1B6885B093F851
:1006100024208DF80B208022ADF804204FF4C06216
:10062000ADF8062061228DF80C2093F84E208DF84D
:100630000E2093F84F20DB698DF80F20002401462F
:100640000093204601236A468DF808408DF80D304E
:1006500002F062FB287088B10521224602F0BCFA44
:10066000009B59060AD540F204412246287802F040
:10067000B3FA28788121224602F0AEFA287805B034
:1006800030BD00BF1882FF1F3484FF1F2DE9F043E7
:10069000564C857B2668A1B0002E34D1402002F054
:1006A0004DFE534B1860582002F048FE514B186025
:1006B0003046FFF725FFB0F5004F07D161204FF41A
:1006C0001661032203F014F8042300E001234A48D2
:1006D000236004F015FB00F08BFD6D20042102F077
:1006E000D1FF0320FFF78EFF00287BD0434B444807
:1006F0001A78444B1A7002F08FFD7520042102F025
:10070000C1FFFFF785FE3D4E384F2846694605225A
:1007100002F078FA58B39DF803309DF8042013B125
:10072000012B18D01EE0032A03D1104604F0B9FAB9
:100730000EE00C2A02D1FFF76BFEE6E7062A05D190
:1007400030783149162202F045FDDEE7832ADCD1FC
:1007500006F0DCFCD9E7DD2AD7D12268082AD4D1FB
:100760003B60D2E72846694602F04CFACDE72368A1
:1007700013F0370F36D0214D287802F053FA88B3A2
:10078000DFF88C80DFF88C902F462878694640226D
:1007900002F038FA044628B3B8F8006006F4804640
:1007A000B6B26846214616B102F0BEF9EDE700F098
:1007B00081F9B9F80020684621467AB901F030FD88
:1007C0000028E2D04FF4807000F0A8FB0228DCD1B2
:1007D00038780E49172202F0FDFCD6E7324601F0C8
:1007E0001FFDD2E721B0BDE8F08300BF1C82FF1FD0
:1007F0001482FF1F1882FF1FE07300003484FF1F64
:1008000050740000FC81FF1F1C7900000579000076
:100810004C82FF1F4082FF1F7047013911F8013FD2
:1008200033B110F9012B5BB29A42F7D00020704728
:1008300090F90020202A07DC03461846013390F97E
:100840000020202AF9D070471846704730B5036859
:1008500002461946013391F90000202803D111689E
:1008600001311160F5E700231846CC5C65B22F2DED
:1008700013DDE5B2A5F13004E4B2092C84BFA5F183
:100880003704E4B2000104F00F0480B2204314687E
:1008900001330134042B1460E7D130BD10B5036877
:1008A00093F90020202A07D01A461346013293F903
:1008B000001031F02004F8D11A46013392F90010EB
:1008C0002029F9D0026092F90000D0F1010038BF70
:1008D000002010BD83885BBA838003681BBA036065
:1008E0007047000008B5054802F096FC044802F085
:1008F00093FC0448BDE8084002F08EBC487E00002E
:10090000408A00005B7E00002DE9F047DFF8D090C0
:100910002D4E99F800204FF00C0808FB02F2B31896
:1009200088B08246B5581F795C7901A820211B2226
:1009300002F016FBBAF1000F04D054450FDD0C3560
:10094000013CFAE7214802F067FC99F8003008FB07
:100950000366B06802F060FC1D4802F05DFC1D4EAD
:100960000C3554B330780021422202F033FC50B9E8
:10097000184B4021187841F26D0202F02DF9164B08
:1009800001201C601CE055F80C0C02F045FCB8423C
:100990000246307802DB01A9012202E0BA1A01A95D
:1009A00092B202F017FC55F8080C02F035FC0B4827
:1009B00002F032FC013C0C35D3E7074B20461C60AB
:1009C00008B0BDE8F08700BFC47D00005A7E00007B
:1009D0005E7E0000FC81FF1F3882FF1F5B7E0000EF
:1009E000EF82FF1F30B587B00446082301A88DF8B9
:1009F000103006F0E7F8A01D02F08DFA0025ADF8E2
:100A000008006571E01C02F086FAA5708DF80A00F6
:100A1000204602F080FA01238DF80B0001A88DF822
:100A2000103006F0CFF8024802F0F6FB07B030BDF8
:100A3000767E000070B51C4D847B8AB00DF10906EE
:100A4000204602A9052202F0DDF858B39DF80B30CC
:100A50009DF80C20012B02D0412B08D01DE0DD2A8F
:100A6000EED128680028EBD0FFF74EFFE8E72046DC
:100A700002A902F0C7F89DF80830042B07D10DF148
:100A800007003146012202F074FA084802E0032B05
:100A9000D6D1074802F0C0FBD2E7204602A902F0F7
:100AA000B1F8CDE70AB070BD3882FF1F857E000027
:100AB000967E00000A46034903460878194602F06C
:100AC00089BB00BF3484FF1F184B194A1B6812688A
:100AD000D8695168884210B50BD1B3F84E00D18E59
:100AE000884206D193F82440117B641A18BF012470
:100AF00000E0012452895B8C53409BB213F0280F15
:100B000018BF44F002045A0748BF44F00404DB064F
:100B100048BF44F008040120FFF7F2FCE00704D5C9
:100B20000420BDE81040FFF76DBD10BD1882FF1F07
:100B30001482FF1F022838B50546184C1AD02168C8
:100B4000182248F2040004F073F8216848F21C00EF
:100B50001831402204F06CF8012D1CD0022004F062
:100B6000A0F80E4B19680E4B18311868402202F09D
:100B700000FA10E00A4B20681B685A89438C5340E6
:100B8000990701D5012038BD0649182202F06FFBF4
:100B90000028D4D0F6E7002038BD00BF1882FF1F20
:100BA0001482FF1F4D84FF1F10B5094C2068FFF70A
:100BB00043FC206807490622023002F0DAF9206877
:100BC000054918304022BDE8104002F0D2B900BFFC
:100BD0001882FF1F3784FF1F107400002DE9F743B0
:100BE0005B4D2B6806460C46032B00F28B80DFE83A
:100BF00003F0022B2685574F3B682BB94FF400704A
:100C0000042102F0BFFB3860534A00231360534AAB
:100C10001360534B3A681A6001232B6014E0514A69
:100C200051480833136004F087F8504B18600223D2
:100C30004F482B6002F0F0FA3846FFF74BFE344481
:100C4000454D1FFA84F954E04548434902680B6852
:100C500040F2FF17BB4224D814B902600B6073E066
:100C600016F801CB0133013C082B02F801CBA4B2EA
:100C7000F0D10B60374B02601F683846FFF72AFE41
:100C8000BA8841F234239A4201D03A4804E03B68E2
:100C9000B3F5003FC3D3384802F0BEFA03232B60FC
:100CA00052E002600B60CAE7B3B299452AD02C4FDC
:100CB0003B685A1C01343A6016F8012B2C60B4F5DD
:100CC000007F1A7015D12D48DFF8888002F0A4FA51
:100CD000264BD8F800101868224604F091F81F4BF4
:100CE0001A6802F500721A6000232B60D8F80030F1
:100CF0003B602C68B4F5007FD6D303E020BB19BB62
:100D0000296021E0154B1449164A1B6809681268CE
:100D10001944914218D305219A428DF80710134CBB
:100D200005D90C4920680968D21A04F069F80DF158
:100D30000701206804F00AF9114802F06DFA6120F9
:100D40002821832202F0D4FC03B0BDE8F08300BF69
:100D50002482FF1F3082FF1FF482FF1F3482FF1F97
:100D60004882FF1F4482FF1FE47E00002C82FF1F89
:100D7000E67E0000B07E0000CA7E0000F47E000027
:100D8000F67E000070B586B00646082301A80C4622
:100D90008DF8103005F016FF96BB6CB33146224635
:100DA0009DF80B0001F0D8FF3A250570024602219C
:100DB0009DF80A00013201F0CFFF0570024631466E
:100DC000BDF80800013201F0C7FF122102469DF86C
:100DD0000D0001F0C1FF0570024602219DF80E00D2
:100DE000013201F0B9FF0246022102F8015B9DF8D1
:100DF0000F0001F0B1FF00E02046001BC0B218E078
:100E0000A01D02F088F800258DF80F006571E01C28
:100E100002F081F8A5708DF80E00204602F07BF8F4
:100E200001238DF80D0001A88DF8103005F0CAFEE1
:100E3000284606B070BD0000F8B51D4B1D4D1E685C
:100E40001423B6FBF3F6B6FBF5F402460021204668
:100E500001F082FF442141706121817005FB14661D
:100E600079214FF461652023B6FBF5F4C170024689
:100E7000732103704371017106322046002101F095
:100E80006BFF05FB14663C253A27B6FBF5F40246DA
:100E9000077002212046013201F05EFF0246077012
:100EA000022105FB14600132BDE8F84001F054BF97
:100EB0006884FF1F8051010038B50F4B1B68D9783B
:100EC0009C789D7901EB0424597902460904D8796C
:100ED00001EB05210144187901EB0060022101F0CA
:100EE0003BFF2D23A4B2024603700A2120460132A3
:100EF000BDE8384001F030BF1882FF1F7FB50648BB
:100F000002F08AF901A8FFF7D7FF01A802F084F9DF
:100F100007B05DF804FB00BF117F0000B0F5807FD3
:100F200010B503460CD0B0F5006F204A11D11288DD
:100F3000002A38D11E4A1288002A34D11D4A0AE0FC
:100F40001C4B1B887BBB194B1B8863BBFFF7A8FAA4
:100F500002E04FF400731380154B1B88B3F5807FBC
:100F600003D12020FFF79CFA09E0124B1A88B2F552
:100F7000006F04D14FF480521A8001F0DFFDFFF7BB
:100F8000BDFFFFF7AFFC0C4802F046F90B4B1868A9
:100F9000393002F041F90024094B20461C70FFF75C
:100FA000B3FC204610BD022010BD00BF2882FF1FE9
:100FB0004082FF1F4C82FF1F237F00001882FF1F0B
:100FC000EF82FF1F313803283FD8DFE800F002111D
:100FD000202F1F4B1F491A6809681868043B1B68BB
:100FE00023EA000001EA02031843C0F340107047EF
:100FF000174B18491A6809681868043B1B6823EAEC
:10100000000001EA02031843C0F380107047104B40
:1010100010491A6809681868043B1B6823EA000035
:1010200001EA02031843C0F3C0107047084B094996
:101030001A6809681868043B1B6823EA000001EA83
:1010400002031843C0F3002070470020704700BF20
:1010500094F00F4080F00F402DE9F843124B1A68CE
:1010600092F85070B2F85280012531200024994640
:10107000461C40B2F6B2FFF7A5FF00B12C436D004D
:10108000392EEDB201D0F0B2F2E7FFF71DFDD9F82D
:10109000003083F8507083F85140A3F8528000204C
:1010A000BDE8F843FFF746BD1882FF1F313803281B
:1010B0001FD8DFE800F0020910170F4B186880F006
:1010C0002000C0F3401070470B4B186880F04000C0
:1010D000C0F380107047084B186880F08000C0F3A0
:1010E000C0107047044B186880F48070C0F3002073
:1010F00070470020704700BF94F00F40303838B57B
:1011000003284AD8DFE800F002090406202405E09D
:10111000802403E04FF4807400E04024642945B249
:101120000AD002DC612938D003E0692904D06F2994
:101130001BD04FF0FF3038BD194B1A6842F40062E3
:101140001A6002202146032206F0ECF8154B1A68BB
:1011500022EA04041C60144B1B68012093F8502001
:1011600000FA05F522EA050515E00D4B1A6842F470
:1011700000621A6002202146042206F0D3F8094BCF
:101180001A6814431C60084B1B68012093F8502018
:1011900000FA05F5154383F85050002038BD00BF14
:1011A0003880044094F00F401882FF1F21B10E4B8D
:1011B0001A6842F400621A6010F0010F14BF202375
:1011C0000023810748BF43F040034207074A1168E4
:1011D00048BF43F08003000748BF43F4807321F405
:1011E000F0710B43136070473880044080F00F406B
:1011F0002DE9F84FB64E336893F8510093F85050EC
:10120000284083F851000121FFF7D0FF012430204E
:10121000B0462C4200F1010614BF6F216921F6B2DD
:1012200040B2FFF76BFF6400382EE4B201D03046C5
:10123000EFE7A84CA84EA94D61235F1C5BB2623B4F
:10124000FFB20E2B09D8DFE803F0162433414F5DBF
:101250006B798795A3CDCDB1BF00236843F480534C
:10126000236003204FF48071042206F05BF82B68A2
:1012700043F480731AE0236843F48053236003200F
:101280004FF40071042206F04DF82B6843F400730C
:101290000CE0236843F48053236003204FF4806103
:1012A000042206F03FF82B6843F480632B6099E03A
:1012B000236843F48053236003204FF40061042229
:1012C00006F030F82B6843F40063EFE7236843F43B
:1012D0008053236003204FF48051042206F022F84B
:1012E0002B6843F48053E1E7236843F48053236081
:1012F00003204FF40051042206F014F82B6843F445
:101300000053D3E7236843F48053236003204FF452
:101310008041042206F006F82B6843F48043C5E7B9
:10132000236843F48053236003204FF400410422D8
:1013300005F0F8FF2B6843F40043B7E7236843F454
:101340000063236002204FF48051042205F0EAFF7D
:10135000336843F4805344E0236843F4006323601C
:1013600002204FF40051042205F0DCFF336843F4FF
:10137000005336E0236843F40063236002204FF4F7
:101380008041042205F0CEFF336843F4804328E017
:10139000236843F40063236002204FF400410422D9
:1013A00005F0C0FF336843F400431AE0236843F4B8
:1013B0000063236002204FF48021042205F0B2FF75
:1013C000336843F480230CE0236843F40063236014
:1013D00002204FF40021042205F0A4FF336843F4F7
:1013E00000233360712F01D0FBB226E7D8F800301C
:1013F0003B4A3C483C493D4CB3F852A010250123E0
:101400004FF400462F464FF4802C4FF400284FF045
:10141000080913EA0A0F70D0802B4CD016D8082B7D
:101420003ED009D8022B35D0042B36D0012B40F00A
:10143000C0804FF4807B3BE0202B34D0402B35D054
:10144000102B40F0B6804FF4805B31E0B3F5006FB5
:101450003BD00CD8B3F5007F2FD0B3F5806F2FD0E1
:10146000B3F5807F40F0A5804FF4805B2AE0B3F5B0
:10147000005F3DD005D8B3F5805F08BFC1F800908C
:1014800097E0B3F5804F35D0B3F5004F08BFC4F8EF
:1014900000808EE04FF4007B0AE04FF4806B07E0A1
:1014A0004FF4006B04E04FF4005B01E04FF4804B1D
:1014B000C1F800B07DE00E607BE04FF4005B01E01E
:1014C0004FF4804BC4F800B073E0266071E000BFB9
:1014D0001882FF1F3880044094F00F40D4F00F4072
:1014E000C8F00F4088F00F40C4F00F4084F00F4068
:1014F0000F605EE0C4F800C05BE0802B49D014D8D8
:10150000082B3BD008D8022B32D0042B33D0012B30
:101510004FD14FF4807B39E0202B32D0402B33D099
:10152000102B46D14FF4805B30E0B3F5006F3AD01A
:101530000BD8B3F5007F2ED0B3F5806F2ED0B3F566
:10154000807F36D14FF4805B2AE0B3F5005F2CD06A
:1015500005D8B3F5805F08BFC2F8009029E0B3F565
:10156000804F24D0B3F5004F08BFC0F8008020E0C2
:101570004FF4007B0AE04FF4806B07E04FF4006B00
:1015800004E04FF4005B01E04FF4804BC2F800B080
:101590000FE016600DE04FF4005B01E04FF4804B6C
:1015A000C0F800B005E0066003E0176001E0C0F895
:1015B00000C05B00013D9BB27FF42BAFBDE8F88F0C
:1015C00010B52B4B1A78110604462FD41A789207BF
:1015D0002ED41A7850072DD41A7891062CD41A7864
:1015E0001B78D20704D513F0400F2249224B1AE092
:1015F000580623D4214B1A78D10721D41A789207A0
:1016000020D41A7850071FD41B7819071ED41B4BFF
:101610001A78D2061CD41A7890061BD41B78184965
:1016200013F0800F174B18BF194614E0164912E04B
:10163000164910E016490EE016490CE016490AE07A
:10164000164908E0164906E0164904E0164902E08A
:10165000164900E0164924B9084601F0DDFD204690
:1016600010BD204601F02CFE001BC0B210BD00BF13
:1016700000F007401C7A0000237A000001F00740C8
:101680002E8A0000EC7C00000C7A00005C790000DF
:10169000017A0000F37C0000AC7B0000FC790000C4
:1016A000D97B0000D07B0000328A0000157A000050
:1016B000807B000038B505F067FC00240546631EFA
:1016C000082B06D8DFE803F007090B0D0F111315DF
:1016D0001700104810E010480EE010480CE01048C9
:1016E0000AE0104808E0104806E0104804E01048FE
:1016F00002E0104800E0104801F08EFDA54202D142
:101700000E4801F089FD0E48013401F085FD0A2CD8
:10171000D5D138BD3B7F0000437F00004C7F0000E7
:10172000557F00005E7F0000677F00006F7F000034
:10173000797F0000837F00008D7F0000977F00008D
:101740001A8100002DE9F0470C468EB01546082896
:1017500000F21E85DFE810F009004200DA02F5020F
:101760001C055C03D4040405A30209B9084605E07E
:10177000042908D101229E4B00201A70FFF7C4F8FB
:10178000044600F013BD052908BF0222F3D0062944
:1017900008BF0322EFD0072908BF0422EBD0092994
:1017A00008BF0522E7D00A2908BF0622E3D00E2988
:1017B00008BF0722DFD00F2908BF0822DBD010297D
:1017C00008BF0922D7D0112908BF0A22D3D0122975
:1017D00040F0DE84864B00201870CFE7029220296B
:1017E00000F2D684DFE811F021003800CB00D404E9
:1017F000B7007A00D404D404D404D404590063009C
:10180000B300D404D404E400C801C801D404D4044F
:10181000D404D404D404D404D404D4042500E400AF
:10182000C801C8013D022D00310005F06FFC00F039
:10183000AFBC704801F0F0FC0020FFF7C1FE00F0E3
:10184000A7BCFFF737FF00F0A3BC92F900003038C7
:1018500005F0F2FB00F09CBC674801F0DDFC674836
:1018600001F0DAFC664801F0D7FC01F0CBFD8221E3
:1018700001F0E3FC634801F0CFFC01F0B7FD8221E9
:1018800001F0DBFC604801F0C7FC01F0A1FD822102
:1018900001F0D3FC5D4800F075BC04A8FFF7CCFA5A
:1018A000002404705A4801F0B7FC04A8F2E1137850
:1018B000313BDBB2032B02D9564800F063BC5648DB
:1018C00001F0AAFC029B93F90000FFF7EFFB04462E
:1018D00008B95248DEE1524800F054BC1078A0F13B
:1018E0003103DBB2032B02D94E4800F04BBC40B2AF
:1018F000FFF7DCFB044610B14B4800F043BC054643
:1019000001263120471C40B2FFB2FFF75BFB08B154
:101910003543EDB27600352FF6B201D0F8B2F1E7DB
:10192000029801F0DCFAC0B2461E02980123184466
:1019300003FA06F6029001F0D2FA01280CBF3543F3
:10194000B543E8B20021FFF731FC00F02FBCFFF7F0
:1019500083FB00F01DBC1378313BDBB2032BC3D8F3
:10196000324801F059FC029B93F90000FFF72AFB73
:10197000044610B12E4800F005BC2E488AE10EAC9A
:10198000104644F82C2D01F0AAFA05462046FEF731
:1019900085FF08B12848F5E3039B05F12F0040B20D
:1019A00093F90010FFF7AAFB002800F0F183F1E79C
:1019B00092F900300BB9102653E0104601F08FFA6F
:1019C0001E4B186002A8FEF769FF029B1A78002AD6
:1019D000F1D002F0DF0252B24C2A01D1042102E020
:1019E000572A2FD10221164A0133116030E000BF7F
:1019F000EF82FF1FA17F0000B57F0000617E000025
:101A0000CC7F0000D97F0000E07F00005B7E0000FB
:101A1000F27F000017800000298000003C80000059
:101A2000458000004D8000005C8000006C8000005C
:101A3000798000007D80000081800000F082FF1F1F
:101A4000F481FF1F422A04D1A34A012111600B44F3
:101A50000293029890F90030002BACD001F05BFAB1
:101A600006469E48DFF870A201F0D6FB20238DF8D1
:101A700010308DF811305746002E40F38983984D71
:101A80008421286801F0D9FB964801F0C5FB0DF1CF
:101A900012084FF01009DAF80020022A06F1FF368A
:101AA00017D0042A28D0012A40F072831B2C07D1BA
:101AB00028680DF1060104F0C9FF9DF8063001E029
:101AC0002B681B783968039341F010019DF80C00D6
:101AD00020E01B2C07D128680DF1060104F0B6FFA9
:101AE000BDF8063001E02B681B883968039341F08C
:101AF0001001BDF80C000DE01B2C04D1286803A9CF
:101B000004F0A4FF02E02B681B6803933968039874
:101B100041F01001C9B201F090FB3B682A680398BC
:101B20001A44022B2A60C3EB090904D0042B0CBF12
:101B30001822002200E00822434498450ED020FAE3
:101B400002F1A1F1200C5FFA8CFCBCF15A0F94BF9A
:101B5000C9B22E2108F8011B083AEEE716B1B9F117
:101B6000000F98D10D221A700A225A7000229A7022
:101B700004A801F051FB7FE792F90030002B00F040
:101B80000783104601F0ABF9112C054601D01D2C3E
:101B900001D1554800E0554801F03EFB02A8FEF790
:101BA0007DFE029B1A78002A00F0F28202F0DF022A
:101BB00052B24C2A01D1042102E0572A04D1022159
:101BC0004B4A0133116005E0422A04D1484A012101
:101BD00011600B44029302A8FEF760FE029801F028
:101BE0007EF9049002A8FEF759FE112C01D01D2C9D
:101BF00006D1029890F9003013B101F08CF900E0A1
:101C000001201C3CE4B23A4F012C8CBF002401247B
:101C10000646B846002E40F3BB823A68022A0AD034
:101C2000042A13D0012A17D1049B14B18DF80C306B
:101C300005E02B7010E0049B34B1ADF80C30284661
:101C400003A904F0B1FE07E02B8005E014B128469B
:101C500004A9F6E7049B2B60D8F80030013E1D4430
:101C6000D8E792F90030002B00F09282104601F084
:101C700036F9044602A8FEF711FE029890F900100A
:101C800011B101F02CF90146204604F073FE044620
:101C900018B9184801F0C0FA88E2174872E211B189
:101CA000012909D074E2154801F0B6FA144B1A88DC
:101CB00042F480421A8079E2114C2388B3F5805FA8
:101CC00001D010485EE2104801F0A6FA238843F4E0
:101CD000005323805CE200BFF481FF1F8980000075
:101CE000F082FF1F9A8000009F800000A680000005
:101CF000F881FF1FAE800000B7800000C7800000A1
:101D00004C82FF1FFF8000001D81000049B10329A4
:101D100040F03E82904B10461C6801F0FCF8208495
:101D200036E28E4D2B88042B05D18D4801F074FAD4
:101D300010232B803AE28B4B08461980FEF7B0FB4C
:101D400034E20492072900F22382DFE801F004283C
:101D50004B5214575C3C04A8FEF778FD044604A8D7
:101D6000FEF774FD0EA9012201F82C0D204602F0A9
:101D70005FFF7D4806E204A8FEF768FD044604A85C
:101D8000FEF764FD0EA9012201F82C0D6FEA444014
:101D90006FEA504080B202F04BFF7448F2E104A8B1
:101DA000FEF754FD03A9012202F063FF002808DBBF
:101DB0006F4801F031FA9DF80C00092101F03DFA5D
:101DC000E6E16C48DEE1644C6B492068182201F0C2
:101DD000D0F82068694B18301968402201F0C9F822
:101DE0006748CFE1FEF7E0FE0020FEF7A3FE65485E
:101DF000C8E1012002F055FF6348C3E1022002F070
:101E000050FF6248BEE10020FEF794FE6048B9E151
:101E10001D2900F2BD81DFE811F01E0065003200CF
:101E200047008200BB01BB01BB01BB01BB01BB0181
:101E3000BB01BB01BB01BB01BB01BB01CF00BB01AF
:101E4000BB01BB0143014301BB01BB01BB01BB01A2
:101E5000BB0157016D01404B4E4F1E6800244FF0EF
:101E6000070808FB0470294601F010FA10B986F83B
:101E700024408AE101340C2CF3D1474882E192F9E5
:101E80000030372B05D1344B1B68DA6942F0010270
:101E900006E0382B06D1304B1B68DA6922F00102CC
:101EA000DA6172E13D486DE12B4B3D4F1E68002425
:101EB0004FF0050808FB0470294601F0E7F960B906
:101EC000F36923F006032CB1012C40F0598143F053
:101ED000020355E143F0040352E10134032CE9D13C
:101EE00030484FE11C4B304F1E68002407EB840044
:101EF000294601F0CBF968B9F369012C23F01803E6
:101F000005D0022C40F03C8143F0100338E143F04F
:101F1000080335E10134032CE8D1244832E10E4BAB
:101F2000234F1E68002407EBC400294601F0AEF9D8
:101F300068B9F369012C23F0600305D0022C40F04E
:101F40001F8143F020031BE143F0400318E10134FB
:101F5000032CE8D1174815E11882FF1F2882FF1FC4
:101F6000348100004C82FF1F40810000528100003C
:101F70006A8100007F8100003584FF1F1482FF1FEB
:101F8000A1810000C2810000E2810000FD8100000B
:101F90001A820000107C00003B83000032820000A7
:101FA000887C0000548300005079000067830000A3
:101FB000AC7D00007D8300007E4C7F4801F02CF951
:101FC0007E4801F029F9236893F824300B2B97BF42
:101FD0007B4A7C48072000FB032001F01DF97A486A
:101FE00001F01AF92368DB69DF074CBF77487848AE
:101FF00001F012F9774801F00FF92368DB699E07B9
:1020000005D413F0040F0CBF0223002300E00123CA
:10201000714A052000FB032001F0FEF86F4801F033
:10202000FBF823686E48DB69DD0654BFC3F3C003C9
:10203000022300EB830001F0EFF86A4801F0ECF8AE
:102040002368DB69580605D413F0200F0CBF002568
:10205000022500E00125644801F0DEF8634800EB4A
:10206000C50001F0D9F8584801F0D6F8002D00F06D
:102070008F805F4801F0D0F82368002193F84E006C
:1020800001F0D2F85B4801F0C7F85B4801F0C4F8F2
:102090002368002193F84F0001F0C6F8554871E01D
:1020A000104600F038FFC0B2632803D8002808BFEC
:1020B000012000E063203F4B1B68152C0CBF83F808
:1020C0004E0083F84F0060E04C4801F0A5F84C4802
:1020D00001F0A2F8012003F01BFF182101F0A4F881
:1020E000484801F099F8002003F012FF182101F090
:1020F0009BF84DE04FF0FF3003F00AFF424841E00B
:102100008C1E082C44D8DFE804F0054310434343F9
:1021100027211800FEF7F2FEFEF7E4FB3B4801F032
:102120007BF8244B186839302CE0224B1868114694
:102130003930142200F01DFF2AE004A90020FEF728
:1021400021FE04A801F068F81F481BE00120114699
:10215000FEF718FE2E4815E01046FEF743FC17E088
:10216000062915D12B48114601F090F8044688B194
:102170002948294601F08AF8044688B1274801E039
:10218000F36102E001F048F802E00420FEF73AFAB9
:1021900000240BE0074B1B685A8C42F0400204E01D
:1021A000044B1B685A8C22F040025A8420460EB021
:1021B000BDE8F0871882FF1F4A820000638200009A
:1021C000107C00006B8200001A8100007482000005
:1021D0007682000078820000887C00005D83000029
:1021E00050790000808200008F820000AC7D0000EA
:1021F0009D820000A9820000AD820000B88200002C
:10220000CD820000DE820000EF820000237F00000C
:102210000A83000019830000208300002883000047
:102220002DE9F04F8E4E8F4C85B0054617468946F6
:102230004FF00008B9F1000F00F00E812A78082A4B
:1022400009D1237823B1013B8748237000F0E4FFD4
:1022500000233370FBE01B2A04D05B2A05D13378BE
:102260001B2B02D132700135F1E033785B2B52D158
:10227000A2F14103032B4ED8DFE803F00E0E080253
:102280002378002B00F0E380013BDFE02378272B4D
:1022900000F2DD800133D9E0DFF800A2DFF8D8B129
:1022A000DAF80020282000FB02B001F015F82A78A7
:1022B0000390412ADAF8002007D10AB9032200E08E
:1022C000013ACAF80020694806E00132032AC8BF73
:1022D00000226748CAF8002000F09EFF039A32B13E
:1022E0006448029200F098FF029A013AF7E76048CA
:1022F00000F092FFDAF80000282202FB00B0029200
:1023000000F08AFFDAF80000029A02FB00B000F049
:10231000E3FF20709BE00A2A00F09980002A00F079
:102320009680DFF878B194F800C0DBF800005249DD
:10233000282303FB00C00A542A780D2A79D10A22E7
:102340000A54384602910193FEF73CF90299DBF8F2
:102350000020019B494803FB021349492278097870
:102360004FF00C0E0EFB01F100EB010E0132D2B268
:1023700050F801809EF805E099180020CDF80CE097
:1023800001F8010C37B93F490988002941D04905B6
:1023900006D53EE0022F03D13B490988002938D0F9
:1023A000002A33D04FF0000C039A624518461AD029
:1023B000D8F800100193CDF808C0FEF72EFADDF82A
:1023C00008C0019B0CF1010C024648B12F48029253
:1023D00000F022FF98F8080098F80910029A09E026
:1023E00008F10C08E0E72A49FEF717FA024668B13F
:1023F00004200921FFF7A6F910B9264800F00CFFC8
:102400003FB9204B1888FEF74BF802E0224800F055
:1024100003FFFEF7EDF8DBF80010124B00221A70F4
:1024200001311E4B0329D4BF19601A604FF0010817
:1024300003E00CF1010C84F800C00A49002333705A
:102440000B78272B05F1010501D92723237009F10A
:10245000FF391FFA89F9EDE6404605B0BDE8F08F77
:102460002082FF1F4E82FF1F4D79000096830000DF
:102470005C7E00009D8000004F82FF1FC47D000035
:10248000EF82FF1F4082FF1F4C82FF1F1A81000056
:102490009A83000085800000818000003C82FF1F3D
:1024A0002DE9F04704460D46164622B1022A00F0F7
:1024B0009E80002060E0C079A379504943EA002360
:1024C0000B8094F90030002B637820DA062B0A8009
:1024D00012D0212B40F08E806279237943EA0223C7
:1024E000474A591E1360022291FBF2F10A31C9B228
:1024F000752000F0ABFE08E0E378222B7AD1414B47
:1025000041491878412200F065FE30462FE00A2B41
:102510002CD002D8092B67D06CE0202B1CD0222BAA
:1025200068D12379617943EA0121354B1960374B32
:102530001E78A3789B074CBF81218221304600F092
:102540004BFBA27812F0010230461ABF8421002210
:10255000882100F041FB09E02D4A1370237962794C
:1025600043EA0222264B06201A6000E00320082DD1
:1025700041D9083DADB20834204B1E889946002E43
:1025800039D0234B1A78202A9A461FD11C4B1F683A
:102590000223013F97FBF3F71E4B072E28BF0726A8
:1025A000072000FB0730B54234BFA846B046C6F14D
:1025B000070318442146424600F0DBFCB04505D332
:1025C00007F114017520C9B200F040FEB9F80020EF
:1025D0000A4B002195428AF8001003D3198003208A
:1025E000BDE8F087551B1D800620BDE8F087002060
:1025F000BDE8F0870420BDE8F08700BFFA82FF1F26
:102600001483FF1F1183FF1F2C8B00003484FF1FD6
:10261000F982FF1F1883FF1F2DE9F043B94E857B18
:102620003378A7B0002B40F09480B74BD3F80080EC
:1026300008F1210000F050FEB44B44001A681ABFA4
:10264000A71CFFB2042799463AB9384600F076FE37
:102650000323C9F8000007704370D9F8003024B193
:10266000023308F12001002002E09C70DC7008E0D9
:1026700011F8012F023322B103F8022C03F8010CE8
:10268000F6E70024A24B8DF812404FF00408012712
:102690004FF0750921460DEB080205200193ADF8B6
:1026A0000E70ADF80A40ADF808408DF814708DF842
:1026B00015808DF8169000F02FFB0823307021460E
:1026C00006AA0520ADF824308DF82A90ADF82240F6
:1026D0008DF826700694ADF81E40ADF81C408DF8BC
:1026E000274000F019FB8B4B069418704023ADF87F
:1026F000243002238DF8273003238DF82630102351
:10270000ADF822304FF48073ADF81C304FF4806385
:10271000ADF81E3021464FF4007306AA0520ADF82F
:10272000203000F0F9FA7C4BADF8224018702146B9
:10273000052006AA8DF826808DF827408DF82A40BE
:102740000694ADF81C40ADF81E4000F0E5FA734B5E
:102750001870734C0DF11D07284606A9052200F0DC
:1027600051FA002800F078819DF81B80B8F1010F24
:1027700039D004D3B8F1750F00F05181ECE723682C
:10278000002BE9D0674B1A6842F480521A60664AFF
:10279000664B1A60664B1A6822F060021A60654B3D
:1027A000654A002119701068997040065CBF0220CC
:1027B000187013689B0602D45E4B17229A705F480C
:1027C0005C49082200F053FD50B1524B594918782A
:1027D000082200F0FFFC59485649082200F0C9FBC6
:1027E0007520012134E19DF81C30CA2B3FD005D85B
:1027F0000A2B00F0E280142B45D0ADE7CB2B18D08C
:10280000CC2BA9D1DFF850914FF000087520C4F807
:10281000008000F0A7FFB9F8003043B1484B1A78A8
:10282000484B40461A70FDF73BFEA9F80080464829
:102830001AE0DFF82481B8F800304BB1404B1A7829
:10284000404B00201A70FDF72BFE0023A8F8003043
:102850004FF000087520C4F8008000F083FF0120CD
:10286000414601F09FFE394800F0D6FC74E7002194
:10287000022001F097FE364800F0CEFCC4F800803C
:1028800075204146E4E033498B7848780A781B0488
:1028900043EA00231343CA7843EA0263B3F5613F76
:1028A00023D8B3F5E13F22D8B3F5614F21D8B3F572
:1028B000164F20D8B3F5964F1FD8B3F5615F1ED8D9
:1028C000B3F5165F4AD8B3F5965F49D8B3F5166FDE
:1028D00048D8B3F5966F47D8B3F5167F46D8B3F509
:1028E000967F94BF0023012341E00C233FE00B239C
:1028F0003DE00A233BE0092339E0082337E00723C2
:1029000035E000BF1183FF1F1482FF1F2083FF1FCC
:10291000A12400001F83FF1F0083FF1FF882FF1FF9
:10292000FC82FF1F388004400301600080C0044027
:10293000D4F00F400183FF1FD0F00F400983FF1F29
:102940003484FF1FFC81FF1FF28A0000FE8A000012
:102950000E8B00001883FF1F4C82FF1F062306E02A
:10296000052304E0042302E0032300E002238A7924
:10297000D01F424242414879012805D0022805D1A2
:1029800042F0020292B201E042F004020979012908
:1029900004D0022904D142F0100201E042F0080202
:1029A00058490968C86981F8243020F01F000243A3
:1029B000CA610420FDF726FECEE6524B1A6892F853
:1029C0002430D2690C2B9CBF4F4951F823104F4B38
:1029D00088BF4FF49641080A1970090C99700021BC
:1029E000D970D1074CBF0721082158709007997101
:1029F00001D5022103E012F0040118BF0121597131
:102A0000110701D5012203E012F0100218BF0222C3
:102A10001A7130783D49072200F0DCFB9CE628461D
:102A200039469DF81C2000F0EDF89DF81D30FE2B76
:102A30007FF492AE364800F0EFFB01219DF81E00B6
:102A400000F0F2FB334800F0E7FB01212160404633
:102A5000022200F04DFE7FE62F4C304E304F2078A2
:102A600000F0E0F8002849D0338813F4C04F22D09A
:102A70005A0416D538780021402200F0ABFB40B153
:102A800006A94022207800F0BDF806A90246387851
:102A90002EE0234B4021187841F2750200F09CF89B
:102AA0002CE006A92078802200F0ACF8014606A8A8
:102AB000FEF794F8D3E706A98022207800F0A2F868
:102AC000054606A92A46207800F084FB338806A82C
:102AD000294602227BB9FFF7A3FB0028BFD04FF4A1
:102AE0000060FEF71BFA0228B9D120780D491722A1
:102AF00000F070FBB3E7FFF793FBB0E727B0BDE84A
:102B0000F08300BF1882FF1F788B00001883FF1F1F
:102B10001B8B0000288B00000083FF1F4C82FF1FCF
:102B20003484FF1FB88B00000A4603490346087827
:102B3000194600F04FBB00BF0083FF1F024B1A78FD
:102B4000024B1A70704700BF0083FF1FFC81FF1FFC
:102B50001223038000487047D08A0000642303805A
:102B600000487047498A0000052803460DD8094AE5
:102B700052F82000027832B9032B08D1064B1868AE
:102B800003780B8070470A8070470020704710461A
:102B9000704700BFB88A00002083FF1F13B5441E92
:102BA0000548E4B200682301C318187B00941C6830
:102BB0000323A04716BDC0462883FF1F08B5044B5A
:102BC0001870000100F0BAFB024B186008BDC04647
:102BD0002483FF1F2883FF1F37B5031C0D1C002013
:102BE000FF2B0CD00648013BDBB2046819016418C6
:102BF000207B0093111C24682A1C0223A0473EBDA1
:102C00002883FF1F13B5441E0548E4B20068230162
:102C1000C318187B00941C680423A04716BDC04647
:102C20002883FF1F13B50749421E0968D2B213015A
:102C3000CB18187B002100921C680A1C0523A047B2
:102C400016BDC0462883FF1F30B50A4B0A4A1B68D1
:102C500014780022A2420BD01D680132854204D1B3
:102C60001D7B8D4201D1D0B203E0D2B21033F1E727
:102C7000002030BD2883FF1F2483FF1FF0B5061CF2
:102C800085B0101C019102920393FFF7DDFF011E36
:102C900001D000203AE0FFF7D7FF071EF9D01C4B08
:102CA000C5181C4B2D011B685D193388002B13D0F0
:102CB000039800F043FB041C68600DD03388181C97
:102CC000009300F03BFB0028E3D0009B2060606095
:102CD000A060C018E060E3827388002B11D00398D5
:102CE00000F02CFB041CA8600BD07688301C00F090
:102CF00025FB0028CDD020606060A0608019E060D6
:102D0000E682029B381C2B60019B2B7305B0F0BD43
:102D1000FFFFFF0F2883FF1F07B5032807D00528F3
:102D200011D0002813D1101C00F074FE10E013899C
:102D300001A80380002343801368064A19781823EA
:102D4000FFF79CFF04E0101C01F090FB00E0002066
:102D50000EBDC046F92F0000F0B50E1C85B0141C46
:102D6000CB0604D52023137004239E430134F307BC
:102D700006D5002804DA2D2323704742013400E0F1
:102D8000071C00230193022333402F4D0393002F90
:102D90002DD0BD4214D9281C0A2104F0E7FA019B6A
:102DA000051C002B04D10128F3D1039B002B01D07B
:102DB000302302E07307ECD5202323700134E8E7C9
:102DC000002D01D001230193291C381C04F0CEFAF8
:102DD000631C0293031CC0B26843303323703F1A54
:102DE0000A21281C04F0C2FA029C051CCFE73027F8
:102DF000201C019B002D09D0002B09D0281C0A2182
:102E000004F0B4FA2770051C0134F1E7002B0DD152
:102E1000730703D52023601C237007E0B30702D596
:102E20003023601C2370302303700130330704D536
:102E30000D2303700A234370023040231E4000D14B
:102E4000067005B0F0BDC04600CA9A3BF7B5CB0688
:102E500002D52023137001324BB2002B04DA302349
:102E6000137078235370023220230B400093082301
:102E70000B404026019307230E4019400F1C0429E4
:102E800000D90427FFB27F000F21141C3B1C8C4685
:102E9000013BDBB2FF2B15D09D00011CE9400D1C4E
:102EA00061460D40291C3031392908D90099002983
:102EB00002D0291C373102E0291C5731C9B22170D8
:102EC0000134E5E7019BD019002B04D00D230370DA
:102ED0000A2343700230002E00D10670FEBD10B5EB
:102EE000031C00229A56202A01D10133F9E7002061
:102EF0000F241A7851B22F290CDDD1B20A1C303AB6
:102F0000D2B200010133092A02D90A1C573A2240E1
:102F10001043EEE710BD10B500220378191C3039BC
:102F2000C9B2092906D9002B18D02D2B00D10122B6
:102F30000130F2E7002301780C1C303CE4B2092C8C
:102F400007D85C00303CDB00E31849B201305B1865
:102F5000F1E7181C002A02D0584200E0181C10BDEE
:102F600000B5031C8218934202D019700133FAE7AE
:102F700000BD10B50023934203D0CC5CC454013390
:102F8000F9E710BDF7B5038A041C0E1C4768151C31
:102F90009A4200D91D1CADB2002D28D0E3687A19E1
:102FA00062609A4215D3DB1B9BB22268E91A009338
:102FB00053186360019102F0F9FB002E12D0391C06
:102FC000009A301CFFF7D5FF009B2168F018019A8A
:102FD00006E002F0EBFB002E04D0301C391C2A1C4A
:102FE000FFF7C7FF02F0DAFB238A5B1B238202F0A4
:102FF000DDFB281CFEBD0000F8B51D1C06AB0F1C38
:10300000161C1C7802F0CAFB052D0DD0062D12D01F
:10301000042D1BD1104B24011B68391C1C1960683E
:10302000321CFFF7AFFF15E00B4B24011B681C1986
:1030300063681C8A0BE0084B24011B681C19636839
:1030400000241A681C829A605A6000E0002402F092
:10305000ADFB201CF8BDC0462883FF1FF7B5041C3C
:10306000151C0F1C02F09AFB218A628AE38A8818D9
:103070004019984202DD5D1AAD1AADB2A168AA18D6
:10308000628201914A19E168A2602E1C8A4205D32E
:10309000D31A2268A3609B1AEE1AB6B202F086FB1E
:1030A0000198391C321CFFF764FFB54204D0B919EE
:1030B000AA1B2068FFF75DFF02F070FB638AA28AFB
:1030C000AB4206D1238AEB189A1800232282A382EE
:1030D00002E0AA18A2825B1B638202F067FB281C35
:1030E000FEBD0000F7B5041C0191002936D102781D
:1030F00043780D1C9A4261D102F050FBA178304B0D
:1031000030481970FFF7A0FD2F49087000280ED035
:103110002E4A2F4B80181B6800011818436820792D
:103120001A8A561D3618D88A864203DD0D7002F0C1
:103130003DFB43E006321A82A11D8C420CD09A68F6
:10314000501C9860207810709868DA68904201D31B
:10315000186898600134F0E706252FE01A4B1E78B6
:10316000002E0DD102784378351C9A4226D18778FB
:103170001448391CFFF768FDFFB2061E06D11DE09A
:103180000F4A177800221A7002F010FB0F4A104BFA
:10319000B6181B6836019E19E3787068032B04D1BA
:1031A000C58A038AED1AADB208E0211C019AFFF727
:1031B00055FF0421051C78B200F064FA281CFEBDFE
:1031C0002683FF1FF92F00002583FF1FFFFFFF0F3E
:1031D0002883FF1F08B5031E04D1081C111CFFF72C
:1031E00081FF05E00020FF2B02D0181CFFF7D6FC62
:1031F00008BD38B5041C031C1A1B0133581E057882
:1032000092B2002DF8D1281C002A03D0081C211CE2
:10321000FFF7E0FF38BD000008B5024B1978FFF753
:10322000E8FF08BDFC81FF1F1FB56A46FFF794FD4C
:103230006846FFF7F1FF05B000BD1FB56A46FFF70E
:1032400005FE6846FFF7E8FF05B000BD07B5031CA3
:10325000002083420AD06A4610705070937011713A
:10326000012368460521D370FFF73CFF0EBD30B542
:103270000023934208D0C45C0133CD18013D2D7862
:10328000A542F6D0012000E0002030BD00B5037853
:10329000002B0FD000228A565BB2934207D0D80F82
:1032A000D1179A42484140420123184307E00130B8
:1032B0000131ECE700200856431E9841404200BD12
:1032C00010B5031C0C78181C1C700A78013352B21C
:1032D0000131002AF6D110BD00B5021C031C981A5A
:1032E0000133591E097849B20029F8D100BD000008
:1032F0000E4B13B500221A800D4B0E4A19600E4B6F
:10330000147819601A1C0378A34203D0002B0CD048
:103310000430F8E74388C9186B461160073355221B
:10332000994202D80A700131FAE713BD3083FF1FBA
:103330002C83FF1F0B82FF1F3483FF1FF8B50E4F36
:103340000E4E3B683488051C1C1903231C4201D017
:103350009C4304340A4A631912689A420AD92A1C07
:10336000201C0021FFF7FCFD3B68201CE31AED1830
:10337000358000E00020F8BD2C83FF1F3083FF1F45
:103380003483FF1FF8B50F4F0F4E3B683488051C80
:103390001C194B1E1C4202D04B421C4064180B4AA5
:1033A000631912689A420AD92A1C201C0021FFF7CF
:1033B000D7FD3B68201CE31AED18358000E00020A3
:1033C000F8BDC0462C83FF1F3083FF1F3483FF1FCF
:1033D000054B00B51A68131C981A0133197880B28E
:1033E0005529F9D000BDC0463483FF1F034B186830
:1033F000034B1B68C01A80B27047C0463483FF1F5E
:103400002C83FF1F044B1868044B1B68C01A044B25
:103410001B88C01A80B270473483FF1F2C83FF1FA4
:103420003083FF1FF0B585B00392574F574A0023F2
:1034300013603B60564B061C1B780C1C2578002D36
:1034400048D06DB29D423ED1221CA31ADBB202933A
:10345000013400256557002DF7D11420584304305E
:10346000FFF76CFF02993860CB43E4182F1C61789A
:10347000002926D049B2331C01911A68002A1ED0B7
:10348000002151568C4601998C4516D1596802602D
:1034900041601A890281002A01D00135EDB25989B3
:1034A00041819A8982819B7BC373002901D1002AC3
:1034B00001D00137FFB2143001E01033DDE70134F1
:1034C000D5E7016008E001340022A256002AFAD1B3
:1034D0000134B3E72F1C02952B4C2368002B47D0F7
:1034E000002F2BD00C207843043080B2FFF726FF4A
:1034F000264E284A2368306094461A68002A19D05C
:103500005A89002A06D0624501D1002159815A8981
:10351000426003E09989002901D04160012241689D
:10352000002901D001214172002A01D003600C3032
:103530001433E2E70C235F43C01B3060039BE818A1
:10354000C0B2FFF73BFB002D12D024682168002990
:103550000ED02389002B09D003200121221CFFF764
:10356000DBFBA073002801D1FF23A3731434EDE724
:10357000094802F003F9094B00221A6002F072FCBC
:10358000029805B0F0BDC0463883FF1F4083FF1F7F
:103590000B82FF1FFFFF00003C83FF1F6884FF1F9B
:1035A000054A06481188CB07DB17034049084B4002
:1035B00098B210807047C0463C83FF1F00B4FFFFE5
:1035C000184B37B51C682368002B29D0E27B0D23EC
:1035D0001A4223D002F0E2F8A389002B02D1E37B48
:1035E000D90716D4237C002B0ED000256A4615700F
:1035F00055702168281C0A7869468A700522CD70AA
:103600000B71FFF7E7FD2574E27B0A23134000D11D
:10361000E37302F0CBF8201C626890471434D2E7C1
:1036200037BDC0463883FF1F38B50C4B051C1C68DE
:1036300002F0B4F80D222368002B0CD0E17B11427C
:1036400007D01B785BB2AB4203D002F0AFF8012089
:1036500002E01434EFE7181C38BDC0463883FF1F62
:1036600000B5074B1B681A68002A07D0127852B2BF
:10367000824201D1D87B02E01433F4E7802000BD00
:103680003883FF1F38B5174B1C682368002B27D0E1
:103690001B785BB2834221D1002918D1124B1D68DF
:1036A000002D14D02B68002B11D09C420DD102F0BC
:1036B00075F8A389002B03D00C4A12689B186B6025
:1036C0000023E37302F072F80AE00C35EAE74A07D8
:1036D00002D5E37B1A0703D4E17301E01434D4E785
:1036E00038BDC0463883FF1F4083FF1F6884FF1F1B
:1036F000F8B5194B0E1C1C68171C002C2BD0174B4F
:103700001D682B68002B26D01B785BB2834220D12A
:103710002368002B1FD09D4219D102F03FF8EB7BAC
:1037200002229343EB732772002F04D1AE81002E47
:1037300004D1667208E0002E00D10126084B1B68F8
:10374000F61801236660637202F030F803E00C346F
:10375000DEE71435D5E7F8BD4083FF1F3883FF1F30
:103760006884FF1F38B5114B1D68002D1DD0104B0C
:103770001C682368002B18D01B785BB2834212D1DF
:103780002B68002B11D09C420BD102F007F80023CC
:103790002B726B72E37B02221343E37302F006F891
:1037A00003E00C35ECE71434E3E738BD4083FF1F3A
:1037B0003883FF1F144A154B11681B680131F0B59F
:1037C000101C1160002B1ED00224082504261A6844
:1037D000002A18D0597A002913D001685F68B942CD
:1037E0000FD1D17B214204D1294200D1D673197A5D
:1037F00011749289002A03D059688A185A6000E02F
:103800005A720C33E3E7F0BD6884FF1F4083FF1F4B
:1038100037B5051C33352B78002B11D0028B8A422B
:103820000ED86A46937001230024D370DD231470F0
:1038300054701371201C69460522FFF7CBFC2C70D5
:1038400037BD0000F0B50B1C34331A7801231A4041
:1038500085B0051C0C1C9446002A05D00A8B0B8DE4
:10386000D31A0B8300230B85271C30373B7898072E
:1038700011D0281C1121DA0700D4132102F03AFEDE
:10388000C0B2002800D094E03B780322934340224A
:1038900013433B708DE020201840029000D085E05B
:1038A000268B002E08D140229343281C3B7002F047
:1038B00011FE201C311C76E0E168E06A0A784005C0
:1038C0001AD50420034202D083433B7014E0201C2D
:1038D000323000780190824206D0201C31300078CE
:1038E000904209D1012E07D004221343221C30320A
:1038F00013700123019A02936046002833D0626955
:103900008B199A4204D8521A92B2002A51D000E080
:10391000321CE38B5B089E420CD9B31A0293264BF0
:10392000A8001858029BC08C834203DB7608B24281
:1039300000D952083B78402003433B70281C02F01A
:10394000CDFF061CE06862698319E360934201D3EE
:10395000A368E3601848AD004359201CD98CFFF7D9
:1039600057FF268525E0111C281C02F0C3FD2368A3
:10397000402101332360231C30331A780A431A7024
:10398000029A002A15D1E36860690133E36083423B
:1039900001D3A268E260238BAD00013B2383064B79
:1039A000201CEB58D98CFFF733FF02E0281C02F0F3
:1039B00091FD05B0F0BDC0465C83FF1F38B5051C06
:1039C0003820FFF7BBFC041E01D100200BE0281CAF
:1039D000FFF7B4FCA0600028F7D043192061E06035
:1039E0006361E583201C38BD10B50C1C083102F062
:1039F000A1FF228B238DD31AC3182383E368181ADF
:103A0000A368E060984202D2E38BC018E060002314
:103A1000238510BDF7B5434E0091017A041C301C7C
:103A2000FFF712F9051C071C002D03D00099490768
:103A300007D476E0291CFFF707F9051C381C002D78
:103A40006FD0394A394BAF181B683F01DF19009B13
:103A50003E609B0707D5E088267AFFF7AFFF344921
:103A6000B6008851B860009A324ED20706D5A088B9
:103A7000FFF7A4FF237A78609B00F050237A2C494B
:103A80009B00CB58002B13D02268DA62237A627B2A
:103A90009B00CB5834331A70237AE0889B00CB58B4
:103AA00064210093E37B584303F072FC009BD884AD
:103AB000237A9B00F358002B2CD0227B33331A70CF
:103AC000237AA188A07B9B00F3580091484364218E
:103AD000019303F05DFC019A64219084237AE07BDA
:103AE0009B00F3580193009B584303F051FC01994C
:103AF0002268C884237A9B00F358DA62237A627BB7
:103B00009B00F35834331A70237AA27A9B00F3583F
:103B100032331A70237A211C3B73207A02F0C8FDDD
:103B2000281CFEBD613D0000FFFFFF0F2883FF1F23
:103B30005C83FF1F4483FF1FF7B5764A8B009C58B8
:103B4000754A01919D58231C3433061C18780227AE
:103B500007400097E36A1BD0E18B0A1C050700D5DC
:103B60004A082769258BB818551920612583DD057A
:103B700001D5013A92B26769B84201D3411A216175
:103B80000198216902F0D8FE238C01332384B8E028
:103B9000802212011A4015D0221C303211780420E4
:103BA0000F1C0740BC4603D081431170009F12E0F8
:103BB000271C32373F78B74202D101431170A8E089
:103BC000674600E0171C190605D5221C313217780C
:103BD000BF1B7A4257412022134223D0132E12D109
:103BE0002B1C34331B78DA0703D50198291CFFF707
:103BF000FBFE2B1C30331A7820210A431A706B68A5
:103C000001336B6085E0112E0CD12B1C30331978F9
:103C1000114200D17DE0914319700198291CFFF7F2
:103C200011FE76E0226801322260D8041AD52A8B70
:103C3000EB8B9A420CD829690E702B696A690133A3
:103C40002B61934201D3AB682B612B8B01332B8308
:103C50002B1C30331A7860231A4203D10198291C97
:103C6000FFF7F0FDE28B238B002F39D19A420BD95D
:103C70002769013323833E7023696069013323611F
:103C8000834201D3A1682161E36A6022134222D0FA
:103C9000271C30373A78D0061DD4218BA28C914254
:103CA00019D399060AD52B1C30331A7802210A43FE
:103CB0001A700198291CFFF7C5FD05E08021EA6A0A
:103CC0000198890002F034FC3B78102213433B70CA
:103CD000636801336360114BE26A1A4211D018E045
:103CE000218C013121849A420BD90133238323692A
:103CF0001E702369656901332361AB4201D3A76854
:103D0000276133342078002803D040B20421FFF724
:103D1000B9FCF7BD4483FF1F5C83FF1F8080000058
:103D20000E4B820010B50C1CD15820220B1C3033D6
:103D3000002C07D01C7814420ED094431C70FFF75F
:103D400081FD09E01C7822431A700B1C34331B7868
:103D5000DA0701D5FFF748FE10BDC0465C83FF1FA0
:103D6000F0B585B003930AAB071C0D1C141C1E781C
:103D700001F014FD03980238082800D93AE103F055
:103D8000EBFA090077009D006A000A013901390148
:103D90003901E5009A4B36011B689E19E90401D5EB
:103DA000B66800E07668002C53D0220605D5381C92
:103DB000211CF26A02F0BCFB4BE063050BD5211C11
:103DC000F26A381C02F076FDC105051CC90F381CCB
:103DD000FFF7A6FF0FE10223E10717D5321C3432AB
:103DE000117819420ED0F28B0B0700D55208F16AF8
:103DF000C90501D5013A92B27284381C316902F0CA
:103E00009BFD08E0381C02F0DFFA04E01C4202D0FF
:103E1000381C02F055FB620703D5381C02F04EFA3D
:103E200004E0230702D5381C02F0C4FAF36AE10665
:103E300003D580225201134303E0A20602D5714A42
:103E40001340F362630604D57F231D40331C3333D4
:103E50001D70B58DCFE06A4B36011B686A4A9E190A
:103E60007368D96A114201D01D8CC4E01D8BC2E079
:103E7000634B36011B689E19B668002D07D1F28B83
:103E8000338BD31A9DB2A34200DBB4E0B2E001F061
:103E90008DFC301C291C221C0830FFF7DFF8051CA4
:103EA00001F07CFC331C30331A7860231A4200D0B6
:103EB000A1E0381C311CFFF7C5FC9CE0504A3601DC
:103EC0001268039693195E68221C301C0830291C66
:103ED000FFF758F8331C34331B78494C19070CD5BD
:103EE000338CDA0709D4F28BB3685208F1689A1858
:103EF000914201D2F26000E0F360F26A6023051C97
:103F00001A427AD0331C30330193197810200142C1
:103F100073D0338BF68CB3426FD8019B81431970F9
:103F200091060DD5039A26680120B618B1680B1CBE
:103F300030331A7802431A70381CFFF783FC5CE0B8
:103F40008021381C490002F0F3FA56E02C4B360170
:103F50001B689E19012C05D9023CB368A4B2002D40
:103F600010D103E07368002D0CD107E0012C05D9B6
:103F70001D605D6073681D605D603CE0A40000250D
:103F8000E55038E0A4001C190023E25CEA54013338
:103F9000042BFAD12EE01A4D36012B68002C02D0EA
:103FA0009E19B3681FE09A1953681024191C303108
:103FB0000878204217D0A04308709168CA6A930617
:103FC00009D50B1C30331A78012002431A70381CB3
:103FD000FFF738FC04E08021381C490002F0A8FA01
:103FE0002B689E1973689A6800251A61DA601D8330
:103FF0001D8400E0002501F0D9FB281C05B0F0BDB0
:104000002883FF1FFFEFFFFF8080000008B5034BF0
:104010008200D158FFF716FC08BDC0465C83FF1F25
:1040200010B5002808D08369581DC27F541C0C327B
:1040300052009B18C477998010BD10B5831CCC0723
:1040400006D50478148040780002044314800232BC
:10405000981C8C0706D51C7814805B781B021C43C7
:10406000148002324B0705D503781380417809028A
:104070000B43138010BD0000F7B5282401935C4367
:10408000364B00901B6800201C19E38A089E83426F
:1040900062D12283131C8A4200D90B1CA28A9FB2D0
:1040A000E382974201D9628200E06382F36800995B
:1040B000658A1960B36880205A6829041043284A29
:1040C00011407268014311605968402251405960A3
:1040D0009968E0684A409A60291CFFF7A1FF009A9E
:1040E0006260E28A638A9A4207D0E368002B06D0B6
:1040F0009B690533DB7F012B01D9E08A2CE0019815
:10410000311C01F01BFF0028F7D17B1B9FB2009BE5
:104110005B190093A38A3D1C9F4200D91D1CF368C4
:10412000009980201960B368ADB25A682904104321
:104130000B4A114072680143116059684022514096
:1041400059609968E0684A409A60291CFFF768FF47
:10415000638AEB186382C4E7FEBDC0467883FF1F05
:104160000000FF03F0B58BB01C1C10AB03900F1CBC
:10417000161C1D7801F012FBA01E042800D995E042
:104180004D4B2D011B685D1903F0DCF8031A67170E
:104190008500F80401D5AB6800E06B68710608D5AE
:1041A0009A69911CC97FC80703D57F210F4001324E
:1041B000D7779B690233DD7F79E06B681D8A76E0F3
:1041C000AC68002C0CD1039805A901F0B7FE251CA2
:1041D00000286CD105A90091381C311C321C37E035
:1041E000A36900250233DB7FDA0760D5AF4206D131
:1041F000E28A238AD31AB34259DB9DB257E001F019
:10420000D5FA391C321C201CFEF728FF061C051CA1
:1042100001F0C4FAA36940270233DB7F3B4246D159
:10422000039805A901F08AFE002840D1A2696168BF
:10423000E0680232431AD17F9BB20F43D777321C1A
:104240009E4200D91A1C92B205AB6068111C009303
:10425000039BFFF711FF051C29E06C68391C321C19
:10426000201CFEF78FFEA36904270233DB7F061CA8
:104270003B421FD001F092FAA3690233DA7FBA43BE
:10428000DA77A169887E01F01DFF0028F9D001F0DE
:104290008DFA301C0EE0002E01D0AB6800E06B6898
:1042A0001A6800259A605A601D8200E0002501F01E
:1042B0007DFA281C0BB0F0BD2883FF1FF0B58BB032
:1042C0006C4626340390201C049105921E1CFEF7B8
:1042D00045FC039C01218C4662426241D2B200231C
:1042E00007926F460578FA8C0195521B92B2FA84B8
:1042F00002924278042A12D0052A23D0022A42D1FF
:104300004379039C1B1B5A425341DBB2002B02D161
:10431000079D002D37D000270123BC4633E0002B3A
:1043200031D0049CFF2C02D08278A2422BD1059D73
:10433000FF2D03D0C2780323AA4224D1002E2CD013
:10434000022320E0002B1ED0002E1CD09D1E6A42AE
:104350005541321C1168002912D08F7884787C4036
:104360007F273C420AD1002D0DD14D7909792D02CC
:10437000294395888D4206D2918004E00832E9E70E
:10438000002D00D010600199029A4018002AA8D18F
:10439000644660426041404230400BB0F0BD37B5EA
:1043A0008369051C0133DB7F002B13D0028A8A420C
:1043B00010D86A46937001230024D370DD23137153
:1043C00014705470201C69460522FEF703FFAB6988
:1043D0000133DC7737BD000070B5041C80780B1CFE
:1043E0007F22011C114028254D430C4E9043E2785A
:1043F000366810436279751926791202324301F04A
:10440000D3FDE278AB1C002A01D1112203E0033571
:10441000EA7F01210A43DA7770BDC0467883FF1F27
:1044200038B5011C7F23194028244C430E4B002231
:104430001B68FF201C19131CE56801F0B5FD002363
:10444000A21CD377621DE382D3779D4203D02B82D7
:104450002B68AB606B60A368002B04D000221A822B
:104460001A689A605A6038BD7883FF1FF7B5051C3B
:10447000294F1C230430A97B284A3C68FEF7FEFB29
:104480000190AE7B2823002E0AD05E43AB89A4198D
:10449000A3826B89D90613D5E31C2022DA770FE0BB
:1044A000687C01305843FEF749FF08238382386057
:1044B000AA7C431C041CDA77301C291C01F042FE44
:1044C000019B17495A18174B12011B689A189368D9
:1044D000E360002B02D09C612B892382AB7BA37607
:1044E000AB7B002B0CD0EB7B002B09D028245C434A
:1044F00039680C19A376A97B231DD977AB89A382D0
:104500005368A360002B03D09C61AA7C631CDA77FC
:104510002D6801982560FEBD7883FF1F654100006E
:10452000FFFFFF0F2883FF1FF0B5151C1C4A85B045
:10453000146828225043241827680E1C002F03D12A
:10454000A068002807D129E0081C1A1C291CB847BC
:10455000072823D1F4E7631CD87F002803D040B29A
:104560000421FFF78FF8A3680234E17FA44601918C
:10457000019C04210C400120002C0FD1DA8A1F8AF3
:10458000D21BAA4206DB181C311C2A1CFEF766FD52
:10459000201C03E0019A63460A43DA7705B0F0BDB8
:1045A0007883FF1FF0B5A1B00E1C80220021051CEE
:1045B0006846FEF7D5FC301CFF2100226B46FFF752
:1045C0007DFE002828D0164F00246B46185900287D
:1045D00023D0002D0BD1002E03D18078FFF720FFD0
:1045E00018E000AA13199988FFF7F6FE12E0827806
:1045F0007F231340282253433A68D3180233022200
:10460000D97F012D01D1A94302E091430A1C012168
:104610000A43DA770834D8E7012021B0F0BDC0465C
:104620007883FF1FF0B5A9B00D1C161C039300245E
:10463000062800D9C2E202F08FFE1301980291020F
:104640000700A002B102B80228255543BD4B1B68E4
:104650005D19EF8AEC68002F1CD1002C00D1ADE26F
:10466000238A002B0FD06268E1688A4202D3E08A75
:10467000121A62606068091A89B20A1C994200D94C
:104680001A1C92B284E0A26940200232D17F814399
:10469000D17792E26B8ABB4200D2A6E0002C00D117
:1046A00082E0238A0593002B00D17DE0A369988BDB
:1046B000591D0490C87F012801DDDA8B9A830138E7
:1046C000C877059B0498A1691A1A92B20B1C049131
:1046D00005332282D87F431C5B005B4240000818F0
:1046E000059300230290191C0598023B834206D0D3
:1046F0000298C018808B8446614489B2F4E78A42EC
:1047000033D1002A4AD1002E04D0AB1CD97F3023EC
:10471000194216D0A98A381C02F032FE002289B252
:1047200091420ED103998B684A68586888210143E9
:104730001160596840225140596099684A409A6016
:1047400001226368E068DF196760874202D3E38A69
:10475000FF1A67600023EB829A421FD1049B40211D
:104760000233DA7F8A43DA7718E06368DF19E36897
:1047700067609F4202D3E08A3F1A67606068511AFF
:104780001B1A9FB28AB2B94200DB3A1C0023EB82AB
:104790000399331C0091111CFFF76EFCA269201CC9
:1047A000118AFFF7FCFD08E2A98A381C02F0E8FD37
:1047B00089B2002916D12B8BBB4205D1002E11D016
:1047C000AB1CDB7FD8060DD403998B684A68586808
:1047D000882101431160596840225140596099680D
:1047E0004A409A600024EC82E8E1FF1AAB8ABFB22B
:1047F0003E1C9F4200D91E1CB6B2002C11D0A369EA
:104800005A1DD17F988B012901DDDF8B9F830139F0
:10481000D177238AA2691B1A2382118A201CFFF7F1
:10482000BEFD039869686A8AC3688A181A6083683B
:10483000426859688020084343493704394001439E
:1048400011609868596840225140424059609A600E
:10485000311C201CFFF7E4FB6B8AF6186E82ACE17A
:10486000384B0C781F6800268021FE828C43012C77
:1048700000D1A6E0022C00D11EE1B44200D064E1D8
:104880006878092800D990E002F05CFD898F8F8F4D
:104890008F4B058F844FE878AA78EE79AB790002C8
:1048A000104336021E43FF22031C802193438900DC
:1048B0008B4216D008D880225200934228D108ADEE
:1048C000281CFEF745F91BE0C02189008B4210D05F
:1048D000C022D20093421BD1039B1C4800930A21A3
:1048E00011E008AD281CFEF739F9039B29880093D5
:1048F00009E008AD1040291CFEF736F900281ED04B
:10490000039A29880092321C0023FFF7B5FB55E17A
:104910003B680424002B00D150E1039A681C118AE3
:104920004BE0AB780398837492E0A978084C0020A0
:104930002170FFF737FE061E0CD0002323700424DD
:104940003CE1C0467883FF1F0000FF03CF8B0000CF
:104950007683FF1F9B4903240B680133DB7F03939E
:10496000002B00D12AE16846A91C01222630FEF75F
:1049700000FB08AF039A7523FB700223BA703B71EA
:10498000301CFE23391C07223E707E707B71FEF7BF
:1049900021FC13E1039B8C480093012103E0039861
:1049A0000221009089480A1CAEE73B680424002BD2
:1049B00000D103E1039A281C118A00229847041CA5
:1049C000FCE06B78A81C04930A2B43D00B2B02D07D
:1049D000002B69D159E07C4F04243B78002B00D197
:1049E000ECE007AC0321221CFFF727FBA578311C64
:1049F000802208A8FEF7B4FA3878291CFF2208ABF9
:104A0000FFF75CFC083608A88319083B1D68002DD9
:104A100003D0A878FFF704FDF4E7A6782478291CD2
:104A20008022FEF79DFA221C3878311C08ABFFF774
:104A300045FC0424002800D1C0E0083508A94B1922
:104A4000083B1868002803D00021FFF7C5FCF4E7F5
:104A50000324B3E05C4F04243B78002B00D1ADE08D
:104A600008AD02212A1CFFF7E8FA387829780122DC
:104A7000331CFFF723FC002800D19FE0039A01219B
:104A8000009203300A1C331C0BE04F4B04241B78AC
:104A9000002B00D192E0039B022100934C48049B21
:104AA0000A1CFFF7E9FA88E03B680424002B00D1D8
:104AB00084E00398018A4EE06978049101293CD88A
:104AC00008AEA81C211C321CFFF7B7FA3E4B1B781E
:104AD000002B03D133880424002B6FD130881F2290
:104AE000282302405A430499BA18023208230129A4
:104AF00013D1D17F194260D099433B68D177002B05
:104B00005BD0C0B207AC207001F0D4F92D4A201C54
:104B1000136800211B68042250E7D27F134006D09F
:104B2000039B022100932B480A1C0023B9E703983A
:104B3000022100900A1C2648B3E73B680424002B9E
:104B40003CD0281C0821032238E73B680424002BB2
:104B500034D0039A118A281C321C2FE7039B1A8A2F
:104B6000002A02D1301C022304E00398291C028A87
:104B70000123301CFFF7D8FC21E703998B7C002B25
:104B800007D0104B1F201B68CC2101331856FEF7AD
:104B90005DFB0020011CFFF705FD0EE0094B1F2007
:104BA0001B68CB210133185605E0064B1F201B68FC
:104BB000CA2101331856FEF749FB0024201C29B0F6
:104BC000F0BDC0467883FF1F7683FF1F7483FF1FED
:104BD000DC8B0000DA8B000028235843034B1B6852
:104BE00018180230C37F1943C17770477883FF1FBD
:104BF0002822034B50431B6818180430C07F7047AD
:104C00007883FF1F094B00B51B68002B0BD01A6877
:104C1000002A06D05A68904201D1986804E0103307
:104C2000F5E7101C00E0181C00BDC0467C83FF1F88
:104C300070B5041C01200E1C151C01F00CFF00288F
:104C400007D101F008FF002800D14120032358407C
:104C5000C0B223B2002B05DA80235B421843C0B2F6
:104C6000032358406404321C2B1C610C01F038FFF4
:104C700070BD03B270B5041C0E1C151C0120002B66
:104C800002DA6404640C002001F0E5FE002805D07F
:104C9000211C321C2B1C01F008FF01E001204042C6
:104CA00070BD08B5022804D003280ED0012817D102
:104CB0000CE0002001F0CFFE002811D080235B42E1
:104CC00018430021C0B20A1C06E0002001F0C3FE18
:104CD000002805D001210022131C01F001FF01E092
:104CE0000120404208BD00B5402801DC303804E016
:104CF000602801DC373800E03D3840B2C0B200BD6A
:104D0000014B18607047C0467C83FF1F38B5094BC4
:104D1000051C1C68002C02D1002009E01034216819
:104D20000029F9D0281C00F048F90028F6D0606866
:104D300038BDC0467C83FF1F10B5041CFFF7E6FF9B
:104D400000280AD100202056FFF7CDFF5C2800D9AB
:104D50005C208C2203039202981810BD37B5051C05
:104D6000FFF750FF0190041E12D1281C01A9042254
:104D700001F06CFE019B002B08D05A1C08D0054A9C
:104D8000551B9D4200D20195019C01E080246401E5
:104D9000201C3EBDFBFF0700F8B5051C0E1C171CB0
:104DA000002809D0FFF7DAFF041D240B8023240319
:104DB0005B01E4182C1901E08C24A4020B4B9C42EB
:104DC00002D90020306010E0201CFFF7C7FF3060E0
:104DD000002806D0201D391C012201F037FE201CBE
:104DE00003E080235B01E418E8E7F8BDFEFF07005D
:104DF00008B501F0BFFD431E9841404208BD0000C8
:104E0000F0B587B00291141C494D00D18DE02E6899
:104E1000002E2CD1471D4748FF2107600822464835
:104E2000FEF79EF86A46301C05A91332FFF7B4FF5F
:104E3000061E53D0059A414BD118090B0903059161
:104E4000B74209D373189F4206D2301CFFF7D0FF38
:104E5000059BA34242D2FF186A46301C05A91332B3
:104E6000FFF79AFF061E39D0B842E3D936E0314841
:104E70003349006882193348531811180919090B6E
:104E80001B0B89B29BB201915C2918D9301C5C2B99
:104E90004CD8802424035C21A41A01910FE0013333
:104EA0008C221F039202284EBF180393B74215D8D5
:104EB000381CFFF753FF002805D1039883B20199EE
:104EC0008B42ECD10AE03B18B34202D980200003A8
:104ED000C01B011D381CFFF78BFFEEE72868022876
:104EE00013D803231B1A261E9E4200D91E1C124BE8
:104EF00005301818321C0299FEF73BF82A68A41BEB
:104F0000B3182B60029B9B190293002C02D10298CC
:104F100000280AD107492A68086802998018221CCB
:104F200001F042FD2B68E4182C60286807B0F0BD42
:104F30008083FF1F8483FF1F8883FF1F04100000EE
:104F400000D0FDFFFFCFFDFFFFFF070073B5124A42
:104F500000241368051C0193201CA3421BD00B786E
:104F60000E4E1460211C221C281C337101F01CFD04
:104F700001A90422301CFDF7FCFF311C0822281C6B
:104F800001F012FD281C211C221C01F00DFDA04285
:104F900000D00194019876BD8083FF1F8883FF1F96
:104FA00008B500F00DFC08BD08B56C20FEF73CFB11
:104FB000002801D101F0D0FE08BD30B50023CA5C45
:104FC0009CB2002A10D0C55654B2A5420AD0602C1B
:104FD00001DD203A02E0402C08DD2032D2B252B28C
:104FE000954203D10133EAE7201C00E0002030BDE8
:104FF0002DE9F043414C424D40F2B3720423571E59
:10500000BFB2BE070ED1A84210D9A0F1F170A0F531
:1050100005400233DBB2062B02D8013292B2EEE732
:10502000073BF7E7A0420AD8002400E00124002251
:10503000DFF8F0C0DFF8CC80DFF8EC900CE000F196
:105040007E4000F5F61000F548600133DBB2062B18
:10505000E3D9073BFAE702226CB1012A0BD148459C
:1050600019D9A0F51810A0F56E501D33DBB2062B30
:10507000F1D9073BFAE71CF8025008FB05F6B042ED
:1050800009D9801B2B44DBB2062B01D9073BFAE779
:105090000132D2B2E0E71B4C0126A0420BD9A0F5A9
:1050A000A8300136A0F5C070F6B20133DBB2062B92
:1050B000F3D9073BFAE70024B0F5616F04D9013456
:1050C000A0F56160E4B2F7E700253C2803D901357B
:1050D0003C38EDB2F9E771B10B4901320A700B4A65
:1050E00016700B4A13700B4B18700B4B1D700B4B4B
:1050F0001C700B4B1F80BDE8F08300BF8033E101C3
:105100000085E201805101001182FF1F0A82FF1F0A
:105110000C82FF1FED83FF1F1084FF1FEC83FF1F16
:105120000E82FF1F068C0000803B26002DE9F04711
:10513000B0F80480042340F2B2740022444504F025
:10514000030617D201344EB902F1F17202F505429D
:105150000233DBB2062BF1D9073BFAE702F1F0721A
:1051600002F5993202F5C0720133DBB2062BE5D9A4
:10517000073BFAE78579DFF8B8C0DFF8B8906C1E16
:1051800054B1013C14F80C7009FB07223B44DBB21C
:10519000062BF5D9073BFAE75EB9022D09D902F5CE
:1051A000A83202F5C0720133DBB2062B01D9073BEE
:1051B000FAE790F807C00CF1FF394B44DBB2062B3D
:1051C00001D9073BFAE7867A477AC47A30B24FEAC8
:1051D000800A8001CAEB00004FF4616A0AFB0700F5
:1051E000DFF850A020440AFB090909EB020079B15D
:1051F000084AA2F80080084A1570084A82F800C0E0
:10520000074A1770074A1670074A1470074A137046
:10521000BDE8F0870E82FF1F1182FF1F0A82FF1F69
:10522000EC83FF1F1084FF1FED83FF1F0C82FF1F05
:10523000068C00008051010070477047704770472E
:10524000704770477047704770470000034B4FF43A
:1052500080421A6000200521FEF76EBC24800040C9
:10526000034B4FF400521A6000200421FEF764BC87
:1052700024800040034B4FF480521A600020032129
:10528000FEF75ABC24800040034B4FF400621A60C2
:1052900000200221FEF750BC24800040034B4FF455
:1052A00080621A6000200121FEF746BC2480004085
:1052B000034B4FF4007200201A600146FEF73CBC1D
:1052C000248000400C4B10B54FF480720B4C1A60D8
:1052D0002368052023F020032360FEF797FE236850
:1052E0009A0607D443F020032360054B1A7842F056
:1052F00040021A7010BD00BF248000400C84FF1FC4
:1053000003B00E400B4B10B580220B4C1A60236883
:10531000042023F010032360FEF778FE2368D906EB
:1053200007D443F010032360044B1A7842F0400284
:105330001A7010BD248000400C84FF1F03A00E4093
:105340000B4B10B540220B4C1A602368032023F04E
:1053500008032360FEF75AFE2368180707D443F0BA
:1053600008032360044B1A7842F040021A7010BD03
:10537000248000400C84FF1F03D006400B4B10B567
:1053800020220B4C1A602368022023F004032360C0
:10539000FEF73CFE23685A0707D443F0040323605A
:1053A000044B1A7842F040021A7010BD248000406D
:1053B0000C84FF1F03C006400B4B10B510220B4C92
:1053C0001A602368012023F002032360FEF71EFE0B
:1053D0002368990707D443F002032360044B1A782B
:1053E00042F040021A7010BD248000400C84FF1F60
:1053F00003B006400B4B10B508220B4C1A60236813
:10540000002023F001032360FEF700FE2368D80785
:1054100007D443F001032360044B1A7842F04002A2
:105420001A7010BD248000400C84FF1F03A00640AA
:1054300038B51C4A1C4D12782B789006DBB211D47B
:105440001A4A12781A4091060CD5194C194B20783B
:105450005B7905211840FEF76FFB2B78DBB21A074A
:1054600048BF22780F4A114C92F90020002A07DB2E
:10547000227822F03F02134202D00520FEF7C6FD3B
:1054800023785D060CD5084A1278540608D5074AD9
:1054900023F040031370084B1A6822F020021A60B0
:1054A00038BD00BF0BB00E4004B00E4003B00E403C
:1054B00007B00E40DC83FF1F0C84FF1F38B51C4A69
:1054C0001C4D12782B789006DBB211D41A4A127850
:1054D0001A4091060CD5194C194B20781B790421E0
:1054E0001840FEF729FB2B78DBB21A0748BF227859
:1054F0000F4A114C92F90020002A07DB227822F093
:105500003F02134202D00420FEF780FD23785D069F
:105510000CD5084A1278540608D5074A23F04003F0
:105520001370084B1A6822F010021A6038BD00BFD1
:105530000BA00E4004A00E4003A00E4007A00E409A
:10554000DC83FF1F0C84FF1F38B51C4A1C4D1278EA
:105550002B789006DBB211D41A4A12781A409106C1
:105560000CD5194C194B2078DB7803211840FEF735
:10557000E3FA2B78DBB21A0748BF22780F4A114CA6
:1055800092F90020002A07DB227822F03F02134222
:1055900002D00320FEF73AFD23785D060CD5084AB9
:1055A0001278540608D5074A23F040031370084BBD
:1055B0001A6822F008021A6038BD00BF0BD00640FE
:1055C00004D0064003D0064007D00640DC83FF1F0E
:1055D0000C84FF1F38B51C4A1C4D12782B7890069E
:1055E000DBB211D41A4A12781A4091060CD5194C24
:1055F000194B20789B7802211840FEF79DFA2B78F2
:10560000DBB21A0748BF22780F4A114C92F90020EA
:10561000002A07DB227822F03F02134202D0022048
:10562000FEF7F4FC23785D060CD5084A1278540680
:1056300008D5074A23F040031370084B1A6822F07C
:1056400004021A6038BD00BF0BC0064004C006400B
:1056500003C0064007C00640DC83FF1F0C84FF1F09
:1056600038B51C4A1C4D12782B789006DBB211D449
:105670001A4A12781A4091060CD5194C194B207809
:105680005B7801211840FEF757FA2B78DBB21A0736
:1056900048BF22780F4A114C92F90020002A07DBFC
:1056A000227822F03F02134202D00120FEF7AEFC26
:1056B00023785D060CD5084A1278540608D5074AA7
:1056C00023F040031370084B1A6822F002021A609C
:1056D00038BD00BF0BB0064004B0064003B0064022
:1056E00007B00640DC83FF1F0C84FF1F38B51D4A3E
:1056F0001D4D12782B7802F02002DBB202F0FF0180
:1057000082B91A4A12781A4090060BD5184C194BD8
:1057100020781B781840FEF70FFA2B78DBB21A07B7
:1057200048BF22780F4A114C92F90020002A07DB6B
:10573000227822F03F02134202D00020FEF766FCDE
:1057400023785D060CD5084A1278540608D5074A16
:1057500023F040031370084B1A6822F001021A600C
:1057600038BD00BF0BA0064004A0064003A00640C1
:1057700007A00640DC83FF1F0C84FF1F064B10B5FB
:105780001C68238841F27B22002B08BF134603804C
:10579000FDF706FF208010BD6C84FF1F72B6024B20
:1057A0001A6801321A6070479883FF1F034A136812
:1057B000013B136003B962B6704700BF9883FF1FB7
:1057C00008B5094B1B88DB070AD5FFF7E7FF074B36
:1057D0004AF202621A804BF280421A80FFF7E6FF1B
:1057E000034B20221A6008BD002005400C20054014
:1057F0008CF00F4008B5054B1A681A60FFF7CEFF12
:10580000FDF7D8FFBDE80840FFF7D0BF0000044017
:10581000F8B52D4E33680446154653B92B4F2C4A24
:1058200027F00107D85B985202333C2BFAD1294B61
:10583000336029480278284B1206FBD51A7812F0FB
:10584000300F1CBF30221A70244B092C1C700BD057
:1058500002D8062C08D01AE0412C11D0432C16D1C6
:105860000A681F4B1A700FE01D4B0A0C1A70062CA9
:105870004FEA112203F8012C03F8021C07D103E0C0
:105880000A68174B1A7002E02B68164A1360FFF77C
:1058900085FF336810489847FFF788FF412C0ED1E9
:1058A000114B1A78013B1B781B0443EA02630D4A33
:1058B000127813430D4A127843EA02232B60064BF9
:1058C000187800F03100F8BD0884FF1FFE81FF1F2B
:1058D000A083FF1FA183FF1F0000024007000240BA
:1058E00006000240080002400B000240090002408E
:1058F000F8B5444B1D68444B1A780132D2B23B2AAA
:105900001A7063D900221A70404B19780131C9B25C
:105910003B29197038D91A703D4B19780131C9B239
:105920001729197024D91A703A4A3B48117803781C
:105930000131C9B211700133DBB2062B01D9073B2B
:10594000FAE71D29037007D1344B1978022903D1D6
:105950000121117003221A70314B1B681B0707D5F8
:10596000304BDC6824B1FFF719FFA047FFF71EFF9B
:105970002B4B1B689F0607D52A4B5C6924B1FFF7A8
:105980000DFFA047FFF712FF254B264C1A6812F0B7
:10599000020F1F4606D0666826B1FFF7FFFEB0472C
:1059A000FFF704FF204A13781E060FD4013BDBB239
:1059B00013703A68D00709D55BB2013306D1246869
:1059C00024B1FFF7EBFEA047FFF7F0FE154B1C6973
:1059D0001E4624B1FFF7E2FEA047FFF7E7FE104B9B
:1059E0001B6859070CD5114B1B689D4208D1B46840
:1059F00034B1FFF7D3FEA047BDE8F840FFF7D6BEAD
:105A0000F8BD00BF00D00340ED83FF1F1084FF1FCF
:105A1000EC83FF1F0A82FF1F0C82FF1F1182FF1FF2
:105A20009483FF1F1484FF1F1082FF1F9C83FF1F9E
:105A30002DE9F84F064690461D460F46FFF7AEFE8D
:105A4000364B374C1A684FF00C0909FB06F94A44EB
:105A5000A260926812F0400F9B4605D105F1100339
:105A6000636005F1140304E005F11803636005F1B8
:105A70001C03DFF8ACA0E3603846D8F804103246C7
:105A80005346FEF7CFFD0328074606D004281BD057
:105A900001282CD1FFF78AFE3CE0DAF80810DAF88A
:105AA00004204B6843F0800313604B6883F040038D
:105AB0004B608B6883F040038B60D8F8003043F074
:105AC0008003C8F8003022E026B984232B61AB6143
:105AD000304609E03046FFF78BF8124B1B6803EBAA
:105AE000401384221A619A610821FFF775F8DBF8E8
:105AF000002002EB090399680B4B0B4021680B4314
:105B000043F080012360C8F8001042F80930FFF725
:105B10004DFE00273846BDE8F88F00BF9083FF1F79
:105B2000F483FF1FF083FF1F0800FF032DE9F047F8
:105B3000AA4E3746AA4DDFF8CC822C7898F8003070
:105B40001C4000F0488134F0080900F08780FFF71E
:105B500025FEE2074AD5A34AA34833232B701378C6
:105B600043F00203137098F8003023F0300388F8F4
:105B700000309E4B19688B6823F040038B60002334
:105B80000B601178137101F0FD0111709849012229
:105B90000A70984A137013711371037003710372C2
:105BA00003730374037503760377137182F830303F
:105BB00082F8343082F838300B7803F0040303F0B5
:105BC000FF08002BF8D18C4B8C4A1B68DFF83CA2F5
:105BD0009A6040321A600420424653464146FEF71E
:105BE00021FD834B8AF812800D221A70A30711D56C
:105BF0003378580703D5824B5A6801325A603B7894
:105C0000990703D57E4B1A6801321A600623337058
:105C100002232B70E2060CD530232B70794B1A78B7
:105C2000002142F020021A7005200A460B46FEF7BA
:105C3000F9FCA3060CD530232B70724B1A78002187
:105C400022F020021A7006200A460B46FEF7EAFCF4
:105C50005FFA89F9FFF7AAFD85F8009024077FF520
:105C60006AAF694A644B1578147818682D0929B20F
:105C700014F0080F00EB4113644C20D08A00090196
:105C8000891A5A4A12681144A1608A68500604D4DD
:105C900003F110026260143303E003F11802626042
:105CA0001C33E360FFF77AFD2A46584B002103209E
:105CB000FEF7B8FCFFF77AFDA27C554B7EE0127828
:105CC00002F0040202F0FF0E22B103F108024FF0CD
:105CD000400E00E01A46C4F800E0D2F800E0CEF32F
:105CE000094CA4F810C00EF03C04042C02D0342C53
:105CF0002BD065E0DFF8F48008018C00041BD8F895
:105D0000000000EB040E8900DEF808E01EF0080F2A
:105D10001CBF005900F080093548415C08BF4FF0B6
:105D20008009C90628464CBF01210221FFF780FEE9
:105D3000D8F800301A59B9F1000F02D022F08002D1
:105D400001E042F080021A5141E000241C619C6194
:105D50002E4CDFF898E024684FEA810C4FEA0118D6
:105D600014F0400FDEF80040CCEB080C6444D4F88B
:105D700008C0284C0CEA040404D1046044F0C004B8
:105D8000846003E0846044F0C0040460880009017A
:105D90000C1ADEF8001021444820486028460021F3
:105DA000FFF746FE012805D0104B1B681A5942F038
:105DB00080021A510B4B1A7802F0DF021A7006E0CB
:105DC00084221A619A6128460821FEF705FF044BD8
:105DD00008221A70AEE6BDE8F08700BF88200740B1
:105DE0008020074094200740D02007409083FF1F69
:105DF000C0200740C4200740F083FF1F8800080030
:105E00002C84FF1F8420074090200740F483FF1F4D
:105E1000982007400800FF03104B1B68403309011E
:105E200043F8202000F1604303F56443C9B21970C0
:105E300020220B4B90FBF2F29200034002F16042F1
:105E4000002B02F5614203DA013B63F01F030133CB
:105E5000012101FA03F31360704700BF08ED00E071
:105E60001F0000800E4B1A6810B542F001020D4C65
:105E70001A60002323600C4B05221A6055200B4A40
:105E80000621FFF7C9FF236843F040032360084B56
:105E900031221A60236843F00103236010BD00BF64
:105EA000388004400000044004000440F55700001E
:105EB00008000440134B20F0800210B51C6851010B
:105EC000000604EB010313D50F48104900680C24A9
:105ED00004FB0200446824F0400444600020186180
:105EE000986111F8223023F0020301F8223010BD2E
:105EF000625822F0040262509A6822F004029A600A
:105F000010BD00BFF083FF1F9083FF1FC02007401C
:105F100008B548B101280AD001300BD10021082270
:105F20000548FDF71DF805E0034B186808BD024B56
:105F3000586808BD002008BD2C84FF1F38B5174BDA
:105F40001D68174B13F820305A070C4624D5154B03
:105F50001B680C2202FB00338B6005EB4015FFF73A
:105F60001DFCA3689B685B0604D405F11003636005
:105F7000143503E005F1180363601C356368E560C0
:105F8000186810F0800403D0FFF710FC022038BD21
:105F9000FFF70CFC204638BD012038BDF083FF1F01
:105FA000C02007409083FF1F2DE9F04F9C46404BD7
:105FB000DFF80C81D3F800900C468B002701FF1A04
:105FC0003C4B1646D3F800A04A0118F8211009EB03
:105FD000020521F00C010AEB070B08F82410FF283A
:105FE0004FF00001A9612961A96085B049F802104C
:105FF000CBF808109B464AF807102F4B06D11A78A9
:1060000022F030021A7008F824104EE093F800A035
:106010004AF0100A83F800A0DBF8003020F0800A74
:10602000BAF1010F3B4402D15960242303E0082157
:10603000596005234821000631D4686880B9664557
:1060400038BF66463046039101920293FDF776F918
:1060500068603046FDF772F9029B019A0399E86087
:10606000164836043040014341F0800021F04001E1
:10607000A86041F0800049F80200DBF800201744D6
:1060800043F0080CB960BAF1000F01D1634603E098
:1060900003F0FB0343F0180308F8243005E0BAF1DD
:1060A000000FF9D043F01003F6E705B0BDE8F08F1C
:1060B000F083FF1F9083FF1F842007400000FF0331
:1060C000C02007401C4B2DE9F0411D6803B205EBD1
:1060D00043159A001C01194BA41A1A68125912F0A0
:1060E000400F0CBF083500262A6808BF402612F072
:1060F0008007984619D16968C2F309420123FEF767
:1061000013FA012814D0D8F800301A1938469168CB
:106110000B4A0A4032431E5906F0800642F08001C5
:10612000324329601A51BDE8F0810120BDE8F081B9
:106130000220BDE8F08100BFF083FF1F9083FF1FA6
:106140000800FF032DE9F0414D4B4E7C1A6842F0E8
:1061500040021A6003F5203301361A6822F08042AB
:1061600042F000421A600B7C012B0C46F6B209D1BA
:10617000444B1A6842F4A0221A605A6C42F005029D
:106180005A6408E0404B1A6842F400521A603F4BD0
:106190004FF4E0621A603E4B1A68102E28BF10269A
:1061A00042F480220C201A607043FDF7C7F8394A88
:1061B000394B1060197841F08001197017461A7830
:1061C0001506FCD4354D02232B704FF4007170017D
:1061D000FDF7D8F8324B334A1860000A107059881E
:1061E0001175D9781176304900220A7028312A7049
:1061F0000A701D460B7803F0040303F0FF06002B22
:10620000F8D10820D5F80080FDF798F8C8F8040008
:106210000820D5F80080FDF791F82B68234AC8F8CC
:106220000C009A6040321A603B684FF008129A6086
:106230001F4B0D221A70ED2203F8B02CFF2203F839
:10624000402CBF2203F8382C49201A4A0621FFF7B8
:10625000E3FD194B8B2203F87C2C062203F8742CE7
:1062600001221E7003F86C2C6389DC0705D50A4BEC
:1062700040221A70102203F8042CBDE8F08100BF00
:1062800000F00140048004403880044068D004409D
:10629000348004409083FF1F0C2107409420074066
:1062A000F083FF1F9C2007409820074088000800CB
:1062B000C02007402D5B0000002107402F4B10B588
:1062C00053F82040052853D8DFE800F003101D2ABA
:1062D00037442B4B1A6842F480621A60294B4FF402
:1062E00040721A602D200C21274A3FE0244B1A6887
:1062F00042F400521A60254B4FF440721A602F206E
:106300000B21234A32E01E4B1A6842F480521A6075
:10631000204B4FF440721A6031200A211E4A25E0BA
:10632000174B1A6842F400521A601C4B4FF440722B
:106330001A60332009211A4A18E0114B1A6842F4F6
:1063400000521A60174B4FF440721A603520082132
:10635000154A0BE00A4B1A6842F400521A60134BBC
:106360004FF440721A60124A37200721FFF754FD9C
:10637000E37843F00803E37010BD00BF308D0000E8
:106380003880044044A00440ED56000000D0044092
:10639000615600000CC00440D555000010D00440E8
:1063A0004955000060D00440BD54000020D0044096
:1063B00031540000034B53F82030DA7802F03702F2
:1063C000DA707047308D00002F4B10B553F8204025
:1063D000052853D8DFE800F003101D2A37442B4B63
:1063E0001A6842F480621A60294B4FF440721A60B6
:1063F0002D200C21274A3FE0244B1A6842F400521A
:106400001A60254B4FF440721A602F200B21234A4B
:1064100032E01E4B1A6842F480521A60204B4FF44F
:1064200040721A6031200A211E4A25E0174B1A6873
:1064300042F400521A601C4B4FF440721A60332031
:1064400009211A4A18E0114B1A6842F400521A60E6
:10645000174B4FF440721A6035200821154A0BE0A3
:106460000A4B1A6842F400521A60134B4FF4407200
:106470001A60124A37200721FFF7CEFCE37843F079
:106480002403E37010BD00BF308D0000388004404D
:1064900040A00440ED56000004D0044061560000C6
:1064A00008C00440D555000014D0044049550000F0
:1064B00064D00440BD54000024D004403154000096
:1064C000034B53F82030DA7822F02402DA70704758
:1064D000308D0000064B53F8203093F90B20002A32
:1064E00005DBDA7802F07F0242F04002DA70704792
:1064F000308D000030B50C4B53F820301A7912F073
:10650000800F4FF001020DD0084C02FA00F01A790A
:10651000DA782568D97162F07F020543DA70256068
:10652000002030BD104630BD308D00000C84FF1FB0
:10653000514B53F8203030B5002B00F09C805A7B33
:1065400011F4C05F02F0F90200F087800C0545D518
:1065500005283AD8DFE800F0030C151E2730474C19
:10656000256845F4806525604FF44075444C2BE068
:10657000424C256845F4005525604FF44075414C68
:1065800022E03E4C256845F4805525604FF4407567
:106590003D4C19E0394C256845F4005525604FF411
:1065A00040753A4C10E0354C256845F4005525609F
:1065B0004FF44075364C07E0304C256845F40055E3
:1065C0002560344C4FF4407525608D0405D54C048E
:1065D0004CBF42F0020242F006025A73CD043CD591
:1065E00005283AD8DFE800F0030C151E27302348B1
:1065F000046844F4806404604FF4407426482BE03F
:106600001E48046844F4005404604FF44074234866
:1066100022E01A48046844F4805404604FF4407443
:106620001F4819E01548046844F4005404604FF40E
:1066300040741C4810E01148046844F4005404609D
:106640004FF44074184807E00C48046844F40054C0
:10665000046016484FF44074046094070BD4C807D4
:1066600003D55A7B42F008025A738A0703D55A7B36
:1066700022F008025A7330BD308D0000388004408B
:1066800008A004400CD0044000C004401CD00440CA
:106690006CD004402CD004400CA0044008D004402E
:1066A00004C0044018D0044068D0044028D00440FE
:1066B000714B2DE9F04105460F4653F8204005285F
:1066C00000F2D880DFE800F00305070C11166B4BD1
:1066D0000CE06A4B0FE0694B1A6842F480520DE0FF
:1066E000664B1A6842F4005208E0654B1A6842F49F
:1066F000806203E0624B1A6842F400621A603B68F1
:10670000580605D528464FF4C0510022FFF710FF68
:10671000012DFB7A06D80B2B0CD85A4A5A4932F86D
:10672000132005E00B2B08D8584A594932F813209A
:10673000CB5C04E00C23EA2201E006237522A3725D
:10674000C2F30423D2B2237062703A68514912F046
:10675000010F02F0060307D07F2048555BB15107B7
:106760004CBF0323022306E0FF2048551BB152070C
:106770004CBF13231223A3707B7BDB0731D5464B21
:106780005E5D730103F1804303F510430022012194
:10679000E01D9980DA809A8218619A61DA600A2293
:1067A00099609A833D4B595D3D4B304653F8252007
:1067B000FFF732FBE37A63F07F03E372394B1A6829
:1067C00042F002021A6006F180466B0006F50436BC
:1067D000033363F07F033370E37863F07F03E37088
:1067E00003E0E37A03F07F03E3727B7B9E073DD5F2
:1067F0002D4B13F805802D4B595D2D4B404653F81A
:106800002520FFF709FBE37A43F02003E372254BD1
:106810001A684FEA481642F0020208F18048013532
:106820001A606D0008F5043365F07F051D70BB88A4
:1068300006F1804606F510469AB2F2820021012246
:106840000734B180F383B282F1803460B2607A7B26
:1068500012F00C0F04D015074CBF06220222B2839F
:1068600000225B42F260B361BDE8F081E37A23F07D
:106870002003E372BDE8F081308D000034800440D5
:1068800028800440668C00007E8C00008A8C00000A
:10689000A28C0000DC83FF1F008C00005A8C0000DB
:1068A000188D00003C800440108D0000608C0000BA
:1068B000E08B0000084B53F82030480703D55A7B83
:1068C00042F001025A730A0703D55A7B22F00102F3
:1068D0005A734FF480707047308D0000114B70B5C3
:1068E00053F82040104B26791D5CE6786B0103F1CC
:1068F000804303F5104326F04006E67094B2DC8234
:10690000DA831960094B01211C6801FA00F0044385
:106910001C60074B186801FA05F5284318601046FB
:1069200070BD00BF308D0000008C00000C84FF1F84
:106930000C800040002070470B4A52F82020D2788B
:10694000520710D4094A125C530103F1804303F546
:1069500010431961064B012101FA02F21968114333
:106960001960FFF731BD7047308D0000108D0000B9
:106970000C80004038B520F4FF64451824F007046B
:10698000092021460022FEF743FF30B92B1BB3F547
:10699000006F03D904F50064F2E7012038BD4FF41D
:1069A0000061FFF7E7BF00002DE9F74F16460F46DD
:1069B000244C51B92368990701D100203EE023F00F
:1069C000030323604FF0040804E020F00303236076
:1069D00000F00308DFF87090DFF868A009F1040BFD
:1069E000C8F10405B54228BF354609EB080318462F
:1069F00039462A460193FCF7BCFA019B2B445B45C0
:106A00002F44C5EB060612D3062021680E4AFEF776
:106A1000FFFE054688B9DAF800300B480433FF2141
:106A20000422CAF80030A846FCF79AFA02E023686C
:106A30001D442560002ED3D1BFE7012003B0BDE87F
:106A4000F08F00BFE883FF1FE483FF1F0346084663
:106A50001946FCF78EBA13B5082204464FF40831E4
:106A60006846FCF786FA009B002C0CBF4FF0FF3401
:106A70004FF05534B3F1553F02D1019BA3420FD0E3
:106A800068464FF40A310822FCF773FA009BB3F111
:106A9000553F07D10198A0420CBF0220002002E020
:106AA000012000E0002002B010BD02280CBF4FF40E
:106AB0000A304FF4083070B5134400F1080404EBB9
:106AC00081049DB293B29D4208D0561C10462146C7
:106AD0000122FCF74EFA04343246F3E7002070BD81
:106AE0002DE9F341050646BF00F07F000125002592
:106AF00044060F46164698460AD54FF40830FFF76D
:106B00004EFF4FF40A30FFF74AFF4FF4083405E018
:106B100002280CBF4FF40A344FF40834B8F1000FC8
:106B200007D004F10803B04403EB87071FFA88F885
:106B300010E055B1B4F5083F14BF4FF408304FF4DE
:106B40000A30FFF72CFF454613E02046FFF727FFEA
:106B50007FB132E0B3B298450BD016F8013B38460E
:106B600063F0FF0301A9042201930437FFF71CFF20
:106B7000F0E701A821460422FCF7FBF9019BB3F1E1
:106B8000553F07D04FF05533204601A90422019309
:106B9000FFF70AFF8DB9043401A821460422FCF74F
:106BA000E8F9019BB3F1553F07D04FF0553320462C
:106BB00001A904220193FFF7F7FE002002B0BDE80F
:106BC000F0810000F8B5037B23F0E003013B0446AD
:106BD000092B00F28A80DFE803F007054D46498A59
:106BE00096233C4100263FE04B4B4C4D1A6842F047
:106BF00000521A604A4B00221A60027B12F0200FEA
:106C00001E4606D000690121FEF7F2F923692B60C8
:106C100003E00121FEF78AFA28601023336064E064
:106C2000404B1B78C372404B1B8883803F4B1B78C3
:106C300083713F4B1B78C3713E4B1B7803723E4BF5
:106C40001B7843723D4B1B788372344B1B68036186
:106C50004BE00021FEF76AFA206146E0006900215E
:106C6000FEF7C6F941E00126013600E000260136B4
:106C7000013600E00026013694F90C30002B08DACA
:106C80002F4B012202FA06F61A6822EA06021A605F
:106C90002BE0214B224D1A6842F000521A602F68F7
:106CA0001E4B17F0010707D000222A601A604FF42C
:106CB00040721A610120F8BD2168224A42F826106C
:106CC0002F6018680121FEF793F91D4B012202FA8B
:106CD00006F61A6832431A6043201B4A0221FFF766
:106CE0009BF81A4A102313602B600020F8BD144B48
:106CF0001A68002122F004021A60FEF717FA144BFA
:106D000000261860B4E7827A124B013A02F03F0283
:106D10001A700026B0E700BF3C80044000D003405A
:106D200014D00340ED83FF1F0E82FF1F1182FF1F4F
:106D30000A82FF1F0C82FF1FEC83FF1F1084FF1FBE
:106D40009483FF1F1484FF1FF15800001CD00340E0
:106D50009C83FF1F1082FF1F774B196810B54C07EB
:106D600040F18780754A1268002A7ED1744A126801
:106D7000500510D5734A107840F0400010707248EA
:106D8000047844F0400404701278D20703D51A68DE
:106D900022F004021A606A4B1B681B0511D56B4B6D
:106DA0001A7842F040021A70694A107840F04000A8
:106DB00010701B78DC0704D55F4B1A6822F00402C0
:106DC0001A605F4B1B68D80411D5624B1A7842F0E9
:106DD00040021A70604A107840F0400010701B7832
:106DE000DA0704D5544B1A6822F004021A60544B97
:106DF0001B689B0411D5594B1A7842F040021A7057
:106E0000574A107840F0400010701B78DC0704D51A
:106E1000494B1A6822F004021A60524B1B6858054D
:106E200011D5514B1A7842F040021A704F4A10782F
:106E300040F0400010701B78DA0704D53E4B1A680A
:106E400022F004021A60474B1B681B0511D5484B02
:106E50001A7842F040021A70464A107840F040001A
:106E600010701B78DC0704D5334B1A6822F004023B
:106E70001A60414B1A7830BF2F4B1B6858070DD44E
:106E80002D4B19602E4B1A6812F4806F1A4620D0D1
:106E90002D4B197801F0BF0119701AE0374B1B78A0
:106EA0009B06EDD5364B374C272018704C20587078
:106EB0002378344813F0200FFAD003785C06FCD511
:106EC0002D4B1A702F4A137803F00C030C2BFAD1B8
:106ED000D6E71368190504D51D4B1A7802F0BF02D6
:106EE0001A70174B1A6812F4805F1A4604D01A4BB6
:106EF000197801F0BF01197013689A0404D5184B72
:106F00001A7802F0BF021A70164B1A6812F4806FDA
:106F10001A4604D0154B197801F0BF011970136897
:106F20001B0504D5134B1A7802F0BF021A70BDE896
:106F30001040FEF73BBC00BF10ED00E00C84FF1FCB
:106F40003480044005A0064000A0064005B006407D
:106F500000B0064005C0064000C0064005D006400F
:106F600000D006402880044005A00E4000A00E403E
:106F700005B00E4000B00E400040064000E0074063
:106F8000044006400640064008B56C20FCF768FB4C
:106F900010F0090046D0244B1B789A0603D5234BEA
:106FA0001B785B0635D4224B1B68580739D51F4B1D
:106FB0001A7812F0470F2ED01B4A1178890604D593
:106FC0001B7803F00703022B27D013781A0705D587
:106FD000164B1B7803F00703032B20D0124B1B78B2
:106FE0009B071ED5114B1B7803F00703042B18D108
:106FF000104B187800F00300022806D0032806D0B2
:1070000001280CBF0720062008BD082008BD092064
:1070100008BD032008BD022008BD042008BD0520CE
:1070200008BD012008BD00BF00E0074001E00740A7
:1070300010ED00E002E0074020F0E003092B5AD8F1
:10704000DFE803F005080C101E252C343E486C20A8
:10705000002152E02A4B00221A700CE0284B00223B
:107060001A7043E0274B1A7842F020021A705A78BF
:1070700042F0C0025A70244B1A6822F0040239E030
:10708000204B1A7842F020021A7082222DE01D4B0C
:107090001A7842F008021A70032226E0194B1A7877
:1070A00042F002021A7020F01F001CE0154B1A7803
:1070B00020F01F0042F002021A7040F0010012E0BE
:1070C000104B1A7820F01F0042F002021A7040F0B4
:1070D000020008E00B4B1A7820F01F0042F0020279
:1070E0001A7040F00300987004225A70064B1A6818
:1070F00042F004021A606C200121FCF7C3BA00BF01
:1071000001E0074000E0074010ED00E0014A024BBB
:107110001A60FEE70400FA050CED00E010B5124A13
:1071200012491348891A00238B4203D01C5CD454A3
:107130000133F9E70F4B104A9342184605D10F4A25
:107140000F490023891A184608E00E490023891ABE
:107150008B42F4D0C45CD4540133F9E78B4202D0A3
:10716000D0540133FAE710BDF081FF1F1282FF1FD8
:10717000508D000010040000100400001482FF1F56
:107180007084FF1FC073000008B5464B1A6842F4B4
:1071900080521A60444A454B1A60454B1A6822F0E7
:1071A00060021A60043B4CF220511B6813F0400F40
:1071B000404B4DF6281219801A800BD04FF4C8723C
:1071C00023F8082C002223F80A2C40F2C11223F8DD
:1071D0000E2C03E0384B4FF4E9721A80374B24220F
:1071E0001A70A02203F8012C354A137813F0020F0D
:1071F000334BFAD01A78D006FCD41A7802F00C027D
:10720000082AFAD12F4B2E4927221A704C225A7085
:107210000B782B4A13F0200FFAD013785906FCD5BF
:10722000294A2A4B1A602A4B28221A70244A1378BA
:1072300003F00C030C2BFAD1264B274A2749136085
:10724000274ADA60274A1A61274A5A61274A9A610F
:10725000274A1A63274A9A60274A9A63274ADA62BA
:10726000274A3C3343F8041F9342FBD1FFF756FFF4
:10727000244B254800221A60FF210422FBF770FEF0
:10728000F9F7CAFA214A224B224823491A60FCF72F
:107290002FF8224822490A22FCF7C4F8FCF790F99B
:1072A000FCE700BF388004400301600080C0044058
:1072B000D4F00F400E20054000200540014006405C
:1072C000064006400440064000001301448004408C
:1072D000004006400080FF1F08ED00E0495200001A
:1072E000395200003B5200003D5200003F52000066
:1072F0004152000043520000455200004752000036
:10730000AC81FF1F00800040E483FF1FFC7F002052
:107310006C84FF1F488D00007084FF1FB08C00003C
:10732000F88B000000F5802049300003012342F46F
:10733000807231B10B421CBF0260994304305B0084
:10734000F7E7704702B4714649084900095C4900F3
:107350008E4402BC704700BF03B471464908400028
:107360004900095A49008E4403BC7047002902D0E5
:10737000B0FBF1F0704708B14FF0FF3000F01EB8DD
:107380000029F8D00246B0FBF1F000FB1121704754
:10739000002902D090FBF1F070470028C8BF6FF0C1
:1073A0000040B8BF4FF0004000F008B80029F4D00A
:1073B000024690FBF1F000FB11217047704700BFBF
:1073C0001000000000000000C0A80003FFFFFF0045
:1073D000C0A80001C0A80001A3483130000000008F
:1073E0006D740000877400007E0400000700000038
:1073F00079740000D8730000040000000001000050
:10740000000000000000000000000000000000007C
:10741000150078002000000017005D000A00000041
:107420000041444D494E002020755461736B6572D4
:10743000264B494E4554495300000000000000000F
:10744000000000000000501403030000325F000041
:107450000D0A0A48656C6C6F2C20776F726C642E75
:107460002E2E204B494E455449530D0A0066617635
:1074700069636F6E2E69636F003947656E6572616F
:1074800074652E62696E000000010001001010009A
:107490000001002000680400001600000028000021
:1074A000001000000020000000010020000000008B
:1074B00000001000000000000000000000000000BC
:1074C00000000000002165F25F2065F1EF2065F209
:1074D000EF2165F22F000000000000000000000016
:1074E000000000000000000000000000000000009C
:1074F000000000000000000000000000000000008C
:1075000000000000002065F2CF2065F1FF2165F248
:10751000FF2065F2FF2065F1AF2166F20F00000049
:10752000000000000000000000000000000000005B
:10753000000000000000000000000000000000004B
:107540000000000000000000002165F24F2065F2FD
:10755000EF2065F1FF2065F2CF2166F20F0CC1FF2D
:107560003F000000000000000000000000000000DC
:10757000000000000000000000000000000000000B
:10758000000000000000000000000000002165F283
:107590000F2065F22F0CC2FF4F0BC1FFEF0BC1FF95
:1075A000FF0CC1FFEF0BC1FF2F0000000000000027
:1075B00000000000000000000000000000000000CB
:1075C000000000000000000000000000002065F145
:1075D0005F2065F1DF1693F85F0BC1FFCF0BC1FF92
:1075E000FF0BC1FFFF0BC1FFFF0BC1FF9F0000009E
:1075F000000000000000000000000000000000008B
:107600000000000000000000002165F29F2065F1ED
:10761000FF2065F1FF2065F1FF2165F2AF0FB2FC9D
:107620005F0BC1FFEF0BC1FFCF11AAFB3F2165F23A
:107630009F2065F25F0000000000000000000000D5
:10764000000000000000000000000000002165F2C2
:107650004F2165F2EF2065F1FF2065F1FF2065F114
:10766000CF000000002165F21F2065F2FF2065F1C8
:10767000FF2065F1FF2065F1CF2165F22F000000AA
:1076800000000000000000000000000000000000FA
:1076900000000000002165F29F2166F22F0CC2FF5E
:1076A0005F0BC1FFEF0BC1FFEF1693F85F2165F28F
:1076B000CF2065F1FF2065F2FF2065F1FF2065F224
:1076C0002F0000000000000000000000000000008B
:1076D0000000000000000000000BC1FF0F0BC1FF05
:1076E000CF0BC1FFFF0BC1FFFF0CC1FFFF0CC1FFA0
:1076F000AF1D72F36F2165F29F2165F20F0000004C
:107700000000000000000000000000000000000079
:107710000000000000000000000000000000000069
:10772000000CC1FF4F0CC1FFEF0BC1FFFF0BC1FFEE
:10773000CF1693F81F2065F23F0000000000000004
:107740000000000000000000000000000000000039
:107750000000000000000000000000000000000029
:1077600000000000000CC1FF0F0CC1FF2F2065F2CC
:107770008F2165F2FF2065F1FF2165F2EF2065F1B1
:107780002F000000000000000000000000000000CA
:1077900000000000000000000000000000000000E9
:1077A00000000000000BC1FF5F0BC1FFEF1693F854
:1077B0005F2065F1CF2065F1FF2065F2FF2065F1C4
:1077C000FF2065F1CF000000000000000000000075
:1077D000000000000000000000000000002065F232
:1077E0003F0CC2FF9F0BC1FFFF0BC1FFFF0BC1FF8F
:1077F000FF0BC1FFAF1D74F45F2165F2EF2165F24D
:107800009F2165F20F000000000000000000000052
:1078100000000000002065F14F2165F2EF2065F2C5
:10782000FF2065F1CF0FB1FC5F0BC1FFEF0BC1FF74
:10783000FF0BC1FFFF0BC1FF9F0000000000000015
:107840000000000000000000000000000000000038
:1078500000000000002065F12F2065F1EF2065F1A8
:10786000FF2065F1FF2065F1FF2165F29F0CC1FF4C
:107870009F0CC2FF2F00000000000000000000006D
:1078800000000000000000000000000000000000F8
:10789000000000000000000000000000002165F270
:1078A0005F2065F1FF2165F2CF2165F22F00000016
:1078B00000000000000000000000000000000000C8
:1078C00000000000000FFF000003FF000081FF0028
:1078D00000C07F0000C03F0000800F0000C1030017
:1078E00000F0010000F8030000FE070000FF0100A7
:1078F00000FF000000FC000000F0070000F00F0097
:1079000000FC3F0000436F6D6D616E64206C696E1A
:107910006520626C6F636B65640D0A00436F6E6E69
:10792000656374696F6E2074696D6564206F75742A
:107930000D0A00005284000055840000001200006F
:10794000658400006A84000002000000082008002E
:1079500031000000312E350032000000556E6465A4
:1079600072766F6C746167650000000052840000DD
:107970005584000000120000408800004988000083
:10798000050000005E880000678800000501000017
:107990007F88000088880000050200009C880000A5
:1079A000A488000005030000BF880000C88800000C
:1079B00005040000E8880000F788000005150000B5
:1079C0001289000020890000051600004F85000084
:1079D0003D890000051100006E85000073850000E0
:1079E000030600001785000001850000000000006C
:1079F000658400006A840000020000004A54414788
:107A000000436C6F636B206C6F737300506F77650E
:107A1000722D6F6E00455A504F52540057616B657E
:107A200075700057616B65757020726573657400C1
:107A3000528400005584000000120000658400009C
:107A40006A84000002000000817F00005789000066
:107A5000000400008B7F00006F890000000500001B
:107A6000957F00008A8900000006000099890000C7
:107A70009B89000000070000B5890000B78900005D
:107A800000090000FF850000D6890000000A000000
:107A900074820000E5890000000E0000768200007C
:107AA000F4890000000F00000F8A0000118A000016
:107AB000001000002C8A0000458400000011000026
:107AC00017850000018500000000000065840000AB
:107AD0006A84000002000000528400005584000007
:107AE000001200004F8500005B85000006020000C8
:107AF0006E85000073850000030600008F8500007E
:107B00009685000003070000AE850000B6850000E2
:107B100003020000CF850000D9850000060A00009E
:107B2000E6850000EF8500000609000001860000E0
:107B30000A860000060800001E8600002686000057
:107B4000011F0000468600004D8600000120000055
:107B5000698600006F860000010000007C8600003E
:107B600085860000011A00001785000001850000CD
:107B700000000000658400006A840000020000002C
:107B80007065726970686572616C206661696C7598
:107B9000726500005284000055840000001200004D
:107BA000658400006A840000020000004578746566
:107BB000726E616C00000000528400005584000069
:107BC00000120000658400006A84000002000000CA
:107BD000536F667477617265004C6F636B757000EC
:107BE0005284000055840000001200001C85000033
:107BF00024850000010A0000388500003F85000050
:107C000001010000658400006A8400000200000099
:107C100033303000000000363030000000003132D8
:107C20003030000000323430300000003438303062
:107C3000000000393630300000003134343030007C
:107C40000031393230300000333834303000003504
:107C50003736303000003131353230300032333099
:107C600034303000528400005584000000120000BF
:107C700017850000018500000000000065840000F9
:107C80006A840000020000004F444400004556454D
:107C90004E004E4F4E4500005284000055840000B7
:107CA000001200007D84000088840000051C000094
:107CB00098840000A4840000051D0000B784000023
:107CC000C284000008000000E8840000F184000085
:107CD0000801000017850000018500000000000079
:107CE000658400006A8400000200000074616D7009
:107CF00065720057444F47005284000055840000CD
:107D0000001200009186000094860000010F000020
:107D1000C1860000C486000001100000F08600004B
:107D2000F386000001110000238700002687000071
:107D3000011B00003E87000041870000011C00007D
:107D4000588700005B870000011D00004C85000083
:107D500070870000011E0000928700009A870000D3
:107D600001020000B8870000C0870000010B00007E
:107D7000DA870000E487000001040000FB870000B0
:107D800006880000010500006E85000023880000C1
:107D9000010C0000178500000185000000000000B4
:107DA000658400006A840000020000004E4F4E45CA
:107DB000000000005254530000000000584F4E00D5
:107DC00000000000487A00000F0C00009E830000B5
:107DD000647C000014030000AD8300006C79000097
:107DE000160C0000C0830000F87C00000F0F00009C
:107DF000D2830000D87A0000110E0000E583000055
:107E0000E07B000011040000F4830000987C000077
:107E10000D07000003840000B87B00000D02000085
:107E200010840000947B00000D0200001D840000FF
:107E3000307A00000F0200002E8400003479000028
:107E40000F02000042840000536F66747761726510
:107E50002076657273696F6E20000A0A0D000A0DA4
:107E60003D3D3D3D3D3D3D3D3D3D3D3D3D3D3D3D42
:107E70003D3D3D0A0D004E657720646174652073B9
:107E800065740D0A000A0D415250207265736F6CC3
:107E90007665640A0D000A0D415250207265736FB9
:107EA0006C7574696F6E206661696C65640A0D009B
:107EB0000D0A42414420464F524D4154202D20711D
:107EC00075697474696E670D0A000D0A4241442099
:107ED0004C454E475448202D207175697474696E65
:107EE000670D0A007A00446F776E6C6F6164696E8B
:107EF000672E2E002A000D0A5465726D696E61743A
:107F000065642C20726573657474696E672E2E2EFD
:107F1000000A0D53657269616C206E756D62657241
:107F20003A2000446576696365206964656E74690A
:107F30006669636174696F6E3A200030203D20529B
:107F4000554E0031203D20574149540032203D20FC
:107F500053544F500033203D20564C505200342093
:107F60003D20564C50530035203D204C4C5300369C
:107F7000203D20564C4C53300037203D20564C4C71
:107F800053310038203D20564C4C53320039203DAF
:107F900020564C4C533300205B6163746976655DF9
:107FA000004C61737420726573657420636175732E
:107FB00065203D20000A0D53797374656D206D6551
:107FC0006D6F7279207573653A0A0D0046726565AA
:107FD0002068656170203D20002066726F6D200072
:107FE0000A0D556E7573656420737461636B203D73
:107FF00020000D0A54686520646576696365206811
:108000006173206265656E206F7065726174696E60
:108010006720666F72200042616420706F72742066
:108020006E756D6265720D0A000D0A506F727420D4
:10803000646972656374696F6E3A20004F555450DD
:1080400055540D0A00494E5055540D0A00496E769C
:10805000616C696420706F72740D0A00506F7274E5
:1080600020697320696E7075740D0A00506F727408
:108070002073746174653A2000310D0A00300D0AD6
:10808000000D0A3F3F0D0A23004D656D6F72792088
:10809000446973706C61790D0A002020202000462D
:1080A000696C6C0D0A0057726974650D0A0045729F
:1080B000617365640D0A00457261736520666169CC
:1080C0006C6564210D0A00436F6E6E656374696EA2
:1080D00067205553422077697468205253323332F7
:1080E000202D20646973636F6E6E65637420555331
:1080F0004220746F20717569742E2E2E0D0A005067
:108100006C65617365207573652055534220636FFC
:108110006E6E656374696F6E21210D0A00506C6587
:1081200061736520737461727420646F776E6C6F15
:1081300061643A000A0D427965204279650A0D00B2
:108140000A0D506172616D65746572207365740A01
:108150000D000A0D54656D702E20506172616D65C1
:10816000746572207365740A0D000A0D50617261A6
:108170006D657465722076616C7565203D20000A1E
:108180000D4E6F2076616C696420706172616D655F
:108190007465727320617661696C61626C650A0D49
:1081A000000A0D4F726967696E616C2070617261BF
:1081B0006D657465727320726573746F7265640A9D
:1081C0000D000A0D466163746F72792070617261EF
:1081D0006D657465727320726573746F7265640A7D
:1081E0000D000A0D506172616D65746572732069CE
:1081F0006E76616C6964617465640A0D000A0D4EE7
:10820000657720506172616D657465727320766167
:108210006C6964617465640A0D000A0D436F6E66D3
:10822000696775726174696F6E2073617665640A3F
:108230000D00496E636F72726563742064617461CE
:10824000206C656E6774680D0A000D0A53657269CB
:10825000616C20636F6E66696775726174696F6EB9
:108260000D0A0042617564203D2000696E76616CE4
:10827000696421003700380020426974730D0A00D8
:108280002073746F70206269742873290D0A004688
:108290006C6F7720636F6E74726F6C200048696733
:1082A000682077617465722000250D0A004C6F7795
:1082B0002077617465722000555342204572726FB9
:1082C0007220436F756E746572730D0A002D204322
:1082D00052432D3136206572726F72733A002D2031
:1082E0004352432D35206572726F7273203A0055E8
:1082F0005342204572726F7220436F756E746572BF
:10830000732072657365740D0A004E657720746979
:108310006D65207365740D0A00656E61626C6500A1
:1083200064697361626C65000D0A496E76616C69FF
:1083300064207377697463680D0A00496E636F7215
:10834000726563742073657269616C207370656512
:10835000640D0A00496E636F727265637420706108
:10836000726974790D0A00496E636F727265637485
:108370002073746F7020626974730D0A00496E6314
:108380006F727265637420666C6F7720636F6E74B2
:10839000726F6C0D0A000A0D0D004D414300202044
:1083A0002020204D61696E206D656E7500204C4166
:1083B0004E20636F6E66696775726174696F6E00D7
:1083C00020202053657269616C20636F6E66696757
:1083D0002E0020496E7075742F4F7574707574205F
:1083E0006D656E750020202041646D696E2E206DD4
:1083F000656E750020202053746174732E206D65A6
:108400006E750020202020555342206D656E75004A
:1084100020202020493243206D656E7500202044C5
:1084200069736B20696E746572666163650046549A
:10843000502F54454C4E455420636F6D6D616E64F2
:10844000730020202043414E20636F6D6D616E6488
:108450007300757000676F20746F206D61696E2006
:108460006D656E750071756974004C656176652087
:10847000636F6D6D616E64206D6F6465007573620E
:108480005F6572726F72730053686F772055534245
:10849000206572726F7273007573625F636E745FD2
:1084A0007273740052657365742055534220636F74
:1084B000756E74657273007573622D736572696190
:1084C0006C0052533233323C2D3E555342206D6F77
:1084D00064652028646973636F6E6E6563742074CD
:1084E0006F207175697429007573622D6C6F6164FA
:1084F000005553422D535720646F776E6C6F616443
:1085000000446973706C6179206D656E75207370BD
:108510006563696669632068656C700075705F7477
:10852000696D650053686F77206F7065726174695B
:108530006E672074696D65006D656D6F72790053AB
:10854000686F77206D656D6F727920757365007344
:10855000686F775F636F6E6669670053686F772037
:10856000636F6E66696775726174696F6E007361BF
:108570007665005361766520636F6E666967757214
:108580006174696F6E20746F20464C4153480072CD
:10859000656A656374005265736574206E6F6E2D35
:1085A0007361766564206368616E676573007265E8
:1085B00073746F726500526573746F7265206661C3
:1085C00063746F72792073657474696E6773007376
:1085D000686F775F74696D6500646973706C617949
:1085E0002074696D65007365745F74696D6500530F
:1085F00065742074696D652030313A32323A35360F
:10860000007365745F646174650053657420446130
:1086100074652032333A30323A3230313000736888
:108620006F775F6C700053686F77206C6F77207086
:108630006F776572206D6F646520616E64206F7066
:1086400074696F6E73007365745F6C70005B6F703C
:1086500074696F6E5D20536574206C6F7720706F46
:10866000776572206D6F6465007265736574005282
:108670006573657420646576696365006C61737405
:108680005F727374005265736574206361757365FE
:10869000006D64004D656D6F727920446973706C74
:1086A0006179205B616464726573735D205B3C6C0F
:1086B0003E7C3C773E7C3C623E5D205B6E756D5D32
:1086C000006D6D004D656D6F7279204D6F64696648
:1086D00079205B616464726573735D205B3C6C3E02
:1086E0007C3C773E7C3C623E5D205B76616C5D004D
:1086F0006D66004D656D6F72792046696C6C205B0C
:10870000616464726573735D205B3C6C3E7C3C7796
:108710003E7C3C623E5D205B76616C5D205B6E75ED
:108720006D5D0073640053746F7261676520446906
:1087300073706C6179207B6173206D647D00736D53
:108740000053746F72616765204D6F6469667920AC
:108750007B6173206D6D7D0073660053746F726171
:1087600067652046696C6C207B6173206D667D00B7
:1087700053746F72616765204572617365205B6138
:108780006464726573735D205B6C656E2D686578DB
:108790005D007365745F6464720053657420706F6C
:1087A00072742074797065205B312E2E345D205BED
:1087B0003C693E7C3C6F3E006765745F6464720098
:1087C00047657420646174612064697265637469CB
:1087D0006F6E205B312E2E345D00726561645F70B8
:1087E0006F7274005265616420706F727420696EDC
:1087F000707574205B312E2E345D0077726974655C
:108800005F706F72740053657420706F7274206FA4
:108810007574707574205B312E2E345D205B302FA3
:10882000315D005361766520706F727420736574DA
:1088300074696E672061732064656661756C74008D
:108840007365745F6261756400536574207365724B
:1088500069616C2062617564207261746500736582
:10886000745F73746F70005365742073746F70203D
:10887000626974732028312F312E352F322900730D
:1088800065745F6269747300536574206461746118
:1088900020626974732028372F3829007365745F4C
:1088A0007061720053657420706172697479202858
:1088B0004556454E2F4F44442F4E4F4E4529007389
:1088C00065745F666C6F770053657420666C6F77B4
:1088D00020636F6E74726F6C2028584F4E2F525465
:1088E000532F4E4F4E4529007365745F6869676862
:1088F0005F77617465720053657420666C6F7720D2
:108900007374616C6C20282529205B312E2E393937
:108910005D007365745F6C6F775F7761746572007B
:1089200053657420666C6F7720726573746172741E
:1089300020282529205B312E2E39395D0053686FA0
:10894000772073657269616C20636F6E6669677505
:10895000726174696F6E00436F6E666967757265E8
:10896000204C414E20696E746572666163650043F8
:108970006F6E6669677572652073657269616C20D8
:10898000696E7465726661636500476F20746F205D
:10899000492F4F206D656E75003400476F20746F4E
:1089A0002061646D696E697374726174696F6E20A1
:1089B0006D656E75003500476F20746F206F7665AA
:1089C00072766965772F7374617469737469637300
:1089D000206D656E7500476F20746F2055534220DF
:1089E0006D656E7500476F20746F20493243206DAE
:1089F000656E7500476F20746F2075744641542072
:108A00006469736B20696E746572666163650039B1
:108A1000004654502F54454C4E455420636C6965B4
:108A20006E7420636F6D6D616E64730061003F3F13
:108A30003F00486F737420646562756767657200F4
:108A400056312E342E303038000902640003010400
:108A50008032090400000103010100092101000026
:108A6000012241000705810308000A080B010202E8
:108A700000000009040100010202000005240000BA
:108A80000205240101000424020205240600010756
:108A900005840340000A09040200020A00000007DE
:108AA000050202400000070583024000000A034D52
:108AB0000061006E00750000B48B0000AD8A0000FC
:108AC000E28A00006D8B00006E8B0000AC8B000012
:108AD00012010002EF020108A21549000001010283
:108AE000030110034D0079002000500072006F0058
:108AF00064005553422052657365740A0D00555346
:108B0000422053757370656E6465640A0D00555399
:108B10004220526573756D650A0D00456E756D6571
:108B20007261746564202800290A0D000501090698
:108B3000A101050719E029E7150025017501950830
:108B400081029501750881019503750105081901D8
:108B50002903910295057501910195067508150087
:108B600026FF00050719002AFF008100C0000A0344
:108B700043006F006E0066002C01000058020000E8
:108B8000B004000060090000C01200008025000051
:108B900040380000004B00000096000000E100009B
:108BA00000C201000084030090D0030008034900C4
:108BB0006E00740004030904436F6D6D616E6420E0
:108BC0006C696E6520626C6F636B65640D0A000AE8
:108BD000060002000000400100000100000000004B
:108BE000B15200009D5200008952000075520000F1
:108BF000615200004D520000015775616D6C00001C
:108C00000304050607081F1C1F1E1F1E1F1F1E1F13
:108C10001E1F48544D004A504700474946004353E1
:108C200053004A530042494E0054585400424D509C
:108C30000049434F003F3F3F0057646F670061703A
:108C400070006D61696E74656E6163650075736255
:108C5000006C6F77506F776572000707070707078B
:108C6000070707070707983A4C1DA60E5307A903E5
:108C7000D4013801EA0075004E00270013000000FF
:108C800000001018100C060402114C1DA60E53070C
:108C9000A903D401EA009C0075003A0027001300E4
:108CA000090000000010180C08061302111800003B
:108CB000398C0000A14F00000000000004000100FA
:108CC0003E8C00008D060000450002000000000000
:108CD000428C0000350A00002500FFFF0000000064
:108CE0004D8C0000192600002500FFFF0000000049
:108CF000518C0000A94F000000000000000001009E
:108D00000000000000000000000000000000000063
:108D1000090A0B0C0D0E0000F5530000B9530000BA
:108D20007D5300004153000005530000C552000070
:108D300000A0064000B0064000C0064000D006403B
:108D400000A00E4000B00E4001000028000000000E
:108D5000FF0000000100000001000000FF00802172
:108D6000017001780906FCD5704701010400B207C3
:028D7000FF0101
:0400000300000410E5
:00000001FF
